:020000040800F2
:1000000038130020D5010008432E00085F2B00089C
:10001000412E0008B9070008F96A00080000000036
:100020000000000000000000000000003D53000838
:100030007B08000800000000CD3000088155000852
:10004000EF010008EF010008BD560008EF010008AD
:10005000EF010008EF0100087D080008EF0100082B
:10006000EF010008EF010008EF010008EF010008B0
:10007000EF010008EF010008EF010008BD070008CC
:10008000EF010008EF010008EF010008EF01000890
:1000900000000000EF010008EF010008EF01000878
:1000A000EF010008EF010008EF010008EF01000870
:1000B000EF010008EF010008EF010008EF01000860
:1000C000EF010008EF010008EF010008EF01000850
:1000D000EF010008DD650008EF010008EF010008EE
:1000E000EF010008EF010008B9330008EF01000834
:1000F000EF0100080000000000000000EF01000810
:10010000EF010008EF01000859480008EF0100085E
:10011000EF010008EF010008EF010008EF010008FF
:10012000EF010008EF010008EF010008EF010008EF
:10013000EF010008EF01000800F002F800F03AF8C3
:100140000AA090E8000C82448344AAF10107DA4532
:1001500001D100F02FF8AFF2090EBAE80F0013F04A
:10016000010F18BFFB1A43F0010318476C70000021
:100170008C700000103A24BF78C878C1FAD85207B2
:1001800024BF30C830C144BF04680C607047000011
:100190000023002400250026103A28BF78C1FBD890
:1001A000520728BF30C148BF0B6070471FB51FBD45
:1001B00010B510BD00F0D2F91146FFF7F7FF06F0B9
:1001C00025FD00F0F0F903B4FFF7F2FF03BC00F0E7
:1001D000F5F900000948804709480047FEE7FEE7B7
:1001E000FEE7FEE7FEE7FEE7FEE7FEE7FEE7FEE7E7
:1001F00004480549054A064B70470000B9560008F7
:10020000390100083809002038130020380B00207D
:10021000380B002053EA020C00F069802DE9F04B06
:100220004FF00006002B1FBFB3FA83F503FA05F465
:1002300024FA05F65E4012BF1643B2FA82F502FABE
:1002400005F4C5F120051EBF22FA05FC44EA0C04A2
:10025000203556EA044C4FEA144418BF641C4FF092
:1002600000084FF00009904271EB030C39D30029CC
:1002700019BFB1FA81F701FA07F6B0FA80F700FA70
:1002800007F6C7F120071EBF20FA07FC46EA0C0656
:100290002037B6FBF4FCA7EB0507103F07F01F0B58
:1002A000CBF120060CFA0BFB2CFA06F644BFB34642
:1002B0000026202FA4BF5E464FF0000B5BEA060C21
:1002C00008BF4FF0010B19EB0B09ABFB027C48EBAD
:1002D0000608C01B06FB02CC0BFB03CC71EB0C0128
:1002E000C1E70B46024641464846BDE8F08B13B5D0
:1002F0004FF000004FF00001AFF30080BDE81C405C
:10030000704710B5431C02E010F8011B71B1810762
:10031000FAD14FF0013202C88C1A8C4314EAC21190
:10032000F9D0C01A0A0603D0C01E10BDC01A10BDF5
:100330000A0401D0801E10BD0902FCD0401E10BD71
:1003400040EA010370B59B072ED14FF00136042A15
:100350002AD308C810C99D1B9D43121F15EAC61554
:1003600017D0D8B2E1B2401A50EA056110D198B264
:10037000A1B2401A50EA05410AD123F07F4024F08F
:100380007F41401A50EA052102D1180EA0EB1460FB
:1003900070BDA342DBD018BA21BA884201D901202E
:1003A00070BD4FF0FF3070BD0AB9002070BD10F86D
:1003B000013B11F8014B63B1A3420AD1521E08D090
:1003C00010F8013B11F8014B1BB1A34201D1521EA1
:1003D000EDD1181B70BD032A40F2308010F0030CE1
:1003E00000F0158011F8013BBCF1020F624498BF88
:1003F00011F801CB00F8013B38BF11F8013BA2F125
:10040000040298BF00F801CB38BF00F8013B11F09F
:10041000030300F07180083AC0F0088051F8043BF3
:10042000083A51F804CBA0E80810F5E7121D5CBFAC
:1004300051F8043B40F8043BAFF30080D20724BFDF
:1004400011F8013B11F801CB48BF11F8012B24BF73
:1004500000F8013B00F801CB48BF00F8012B7047C2
:100460004FF000020429C0F0128010F0030C00F0DD
:100470001B80CCF1040CBCF1020F18BF00F8012B5B
:10048000A8BF20F8022BA1EB0C0100F00DB85FEA29
:10049000C17C24BF00F8012B00F8012B48BF00F8F5
:1004A000012B70474FF0000200B513469446964664
:1004B000203922BFA0E80C50A0E80C50B1F1200177
:1004C000BFF4F7AF090728BFA0E80C5048BF0CC025
:1004D0005DF804EB890028BF40F8042B08BF704783
:1004E00048BF20F8022B11F0804F18BF00F8012BF5
:1004F000704770477047704710B5203AC0F00B80C6
:10050000B1E81850203AA0E81850B1E81850A0E817
:100510001850BFF4F5AF5FEA027C24BFB1E8185071
:10052000A0E8185044BF18C918C0BDE810405FEAE1
:10053000827C24BF51F8043B40F8043B08BF70475D
:10054000D20728BF31F8023B48BF11F8012B28BF62
:1005500020F8023B48BF00F8012B7047754600F0B9
:1005600029F8AE4605006946534620F00700854647
:1005700018B020B5FFF73CFEBDE820404FF0000664
:100580004FF000074FF000084FF0000B21F007017B
:10059000AC46ACE8C009ACE8C009ACE8C009ACE8BE
:1005A000C0098D4670470446AFF300802046FFF730
:1005B0000AFE000000487047D408002001491820B6
:1005C000ABBEFEE7260002007047000070B586B0A3
:1005D000044614216846FFF765FF022002F0D4FAB2
:1005E0000C4E0D4D694636F8140000900120019024
:1005F000002002900220039055F8240000F0E6FB52
:1006000036F8141055F82400002200F097FC06B0CC
:10061000002070BD7071000880000020054910B5F1
:10062000054A31F8101052F8200000F07FFC00203D
:1006300010BD0000707100088000002070470000AD
:1006400030B585B00D46044614216846FFF72AFFF1
:100650001CB1012C01D0022C02D1012002F094FA2D
:100660001D4830F8140000900120029002200390F1
:100670001A484DB34FF40411019150F82400694613
:1006800000F0A4FB1448801D50F82410144800EB1F
:10069000C400054600F0E3FA104800210C3050F881
:1006A0002420284600F0E1FA0C480B4D18300A3D92
:1006B00050F824102857002200F088FC285700F03A
:1006C00077FC05B0002030BD0021019150F82400D6
:1006D000694600F07BFBF4E7767100088C0000208F
:1006E000BC08002070B54FF090444FF4807530B1D5
:1006F000012806D0022810D003280CD10DE00022DA
:100700000CE000220221204600F018FC01222946BC
:10071000204600F013FC002070BD0122022120467B
:1007200000F00CFC0022F2E708B1162070470F2001
:1007300070470220704730B585B014216846FFF736
:10074000B1FE012002F02AFA012002F027FA4FF44C
:1007500080740120CDE900400020029003204FF07A
:10076000904503906946284600F030FB0222694616
:100770002846009200F02AFB00222146284600F07D
:10078000DDFB00220221284600F0D8FB05B0002046
:1007900030BD012070470020704710B50020FFF7E2
:1007A0004DFF10BD10B50120FFF748FF10BD10B57B
:1007B0000220FFF743FF10BDFEE70000014800F0F4
:1007C00031B900008401002030B5416C036821F08C
:1007D00003020E4CD9B214250839A34205D2B1FB4D
:1007E000F5F10B4B1A44826406E0B1FBF5F1084BBE
:1007F0001C331A44C91D8264054A8032C26401F068
:100800001F0201219140016530BD00000804024033
:10081000000802400179084A01F07F0102EB8102E1
:100820004265054A4432491E826501F003020121F6
:100830009140C16570470000FC08024030B5D0E926
:1008400013456560446D14B1D0E91645656090F8B4
:10085000444004F01C050124AC40056C6C60046845
:1008600063608368102B036803D099600068C260DE
:1008700030BD9A600068C16030BD7047012000F053
:1008800099BA72B6FEE70000034988688A68824216
:10089000FBD1C043704700000028004010B540B1B4
:1008A00090F825100022022905D00421C16380F8A8
:1008B0002420012010BD01680B6823F00E030B609B
:1008C000816C0B6823F480730B6001680B6823F064
:1008D00001030B6090F84410012301F01C0403FA9B
:1008E00004F1046C6160D0E913144C60416D31B1C6
:1008F0000C6824F480740C60D0E916144C6080F805
:10090000253080F82420002010BD10B590F8251067
:100910000024022903D00421C16301242BE00168D3
:100920000A6822F00E020A6001680A6822F00102D9
:100930000A60816C0A6822F480720A6090F84410A0
:10094000012301F01C0103FA01F2016C4A60D0E9B5
:1009500013124A60416D31B10A6822F480720A6054
:10096000D0E916124A6080F82530002180F8241062
:10097000816B01B18847204610BD000070B50400AE
:1009800011D02068016821F001010160224A20682D
:100990001421904209D2214A0244B2FBF1F18900AC
:1009A00061641F490AE0012070BD1B4A52420244A3
:1009B000B2FBF1F18900616417490839002521640F
:1009C000056094F8440000F01C0101208840216C6F
:1009D00048602046FFF7F8FEA06C0560D4E91301DB
:1009E00041606068401E032807D82046FFF712FFC9
:1009F000606D0560D4E9160141606565A565E56532
:100A0000E56225636563A563E56384F8255084F892
:100A10002450002070BD000008040240F8FFFDBF14
:100A200000000240F0B4016C0B6801680A6890F89D
:100A30004440042604F01C0406FA04F51D4212D0BA
:100A4000550710D50A68920603D40A6822F00402FA
:100A50000A6090F8441001F01C0106FA01F5016CDF
:100A60004D60016B26E0022505FA04F71F424FF0A6
:100A7000000C4FF0010621D097071FD50A68920697
:100A800005D40A6822F00A020A6080F82560194A33
:100A90000168914290F8441001F01C0105FA01F53B
:100AA00002D915490D6002E0124980394D6080F885
:100AB00024C0C16A00291AD0F0BC08470825A54007
:100AC0001D4214D0120712D50A6822F00E020A60E5
:100AD00090F84410026C01F01C0106FA01F151601B
:100AE000C66380F8256080F824C0416BE2E7F0BC63
:100AF00070470000800002400404024070B504000A
:100B00000CD02D4A20681421904209D22B4A02446D
:100B1000B2FBF1F18900616429490AE0012070BD4E
:100B2000254A52420244B2FBF1F189006164224934
:100B300008392164022184F82510016847F6F07213
:100B400091430160D4E902100143D4E90402104347
:100B50000143A0690143E0690143206A0143206821
:100B60000268114301602046FFF72EFEA0680025B1
:100B7000B0F5804F00D165602079A16C00F07F0056
:100B80000860D4E9130141606068401E032808D85A
:100B90002046FFF73FFE606D0560D4E91601416015
:100BA00002E06565A565E565E563012084F825003B
:100BB00084F82450002070BD08040240F8FFFDBFF7
:100BC0000000024070B5044690F82400002501287A
:100BD0000ED0012084F8240094F825600020012E16
:100BE00008D08021E16384F824000125284670BDE7
:100BF000022070BD022684F82560E0632068066844
:100C000026F0010606602046FFF718FE206B00283C
:100C10002068016802D041F00E0106E021F00401D5
:100C200001602068016841F00A010160A06C016860
:100C3000C90303D5016841F480710160606D18B18A
:100C4000016841F4807101602068016841F0010190
:100C50000160CBE711B4009818BC04F070BD10B16E
:100C6000016000207047012070470346002009B151
:100C7000012070475A6070472DE9F04F0022DFF8DD
:100C8000D8904FF0070A4FF0010B60E00BFA02F723
:100C900017EA01035AD022F003054D44AC689607C9
:100CA0004FEA167C0AFA0CF606EA0408B0F1904FF7
:100CB00004D02A4CA04203D1012407E0002405E01F
:100CC000274CA04201D1022400E0072404FA0CF4CE
:100CD000444520D1DFF88CC0DCF800409C43CCF8C0
:100CE00000400CF1040CDCF800409C43CCF80040C0
:100CF000DFF870C0ACF1800CDCF800409C43CCF80D
:100D000000400CF1040CDCF800409C43CCF800409F
:100D1000AB68B343AB60046855000323AB401C438E
:100D20000460D40800EB8404256A56074FEAD66CA9
:100D30000F2606FA0CF6B543256284689C4384604E
:100D40004468BC434460C4689C43C460521C31FA8C
:100D500002F39BD1BDE8F08F000001400004004881
:100D6000000800488008005810B5012801D009A3E8
:100D700009E00020FFF752FC1420FFF76BFF002072
:100D8000FFF74CFC07A30022BDE8104011461046B7
:100D900005F02ABC556E6B6F6E7720427574746FC8
:100DA0006E0D0A00425554544F4E205357310D0AD0
:100DB00000000000044910B50A68024202D0086031
:100DC000FFF7D2FF10BD00000C0800582DE9F04FCE
:100DD000DFF848A1DFF844810AF1800A00224FF0D1
:100DE000010E4FF0030C08F104090AF1040B8DE029
:100DF0000EFA02F52B407DD00C7904F00304012C8F
:100E000001D0022C10D1866854000CFA04F7BE43BE
:100E1000CF68A740374387604468AC430D79C5F37A
:100E200000159540254345600C79E443A40708D09C
:100E3000C56854000CFA04F6B5438E68A6402E43EC
:100E4000C6600C7904F00304022C0CD1D40800EB2A
:100E50008406356A5407E40E0F27A740BD430F6987
:100E6000A7402F433762056854000CFA04F6B543D7
:100E70000E7906F00306A6402E4306604C6814F473
:100E8000403F42D0264C22F003052F19BD6894073D
:100E9000260F0724B440A543B0F1904F04D0214C55
:100EA000A04203D1012407E0002405E01E4CA0422B
:100EB00001D1022400E00724B4402C43BC60D8F8E0
:100EC00000404D689C43ED0200D51C43C8F800402B
:100ED000D9F800404D464E689C43B60200D51C43ED
:100EE0002C60DAF8004055464E689C43F60300D566
:100EF0001C4300E009E02C60DBF800405D464E68D2
:100F00009C43B60300D51C432C60521C0B6833FA7B
:100F100002F47FF46DAFBDE8F08F000000080058C8
:100F2000000001400004004800080048426921EA2E
:100F300002030A4043EA0241816170470AB18161BC
:100F4000704781627047000003490020097800293A
:100F500001D004F029BC70470000002010B5002427
:100F6000032000F053F800F091FA064908600F20C2
:100F700000F00AF808B1012401E000F007F820466B
:100F800010BD00003000002000207047704700288E
:100F90000DDB00F01F02012191404009800000F1AB
:100FA000E020C0F88011BFF34F8FBFF36F8F704701
:100FB000002809DB00F01F02012191404009800058
:100FC00000F1E020C0F8001170470000F0B40E4BB3
:100FD0001B68C3F30223C3F10704042C00D90424C3
:100FE0001D1D072D01D2002300E0DB1E012606FA9D
:100FF00004F56D1E0D409D409E40761E164045EA4C
:101000000601F0BC05F079BD0CED00E0064A00F0E9
:10101000070110684FF6FF03184040EA012003491A
:1010200008431060704700000CED00E00000FA0576
:101030000D48016821F4804101600C4832210068AC
:1010400048430B49B0FBF1F00749143100E0401E62
:101050000A68920501D50028F9D10868800501D5F4
:101060000320704700207047000400583000002023
:1010700040420F000248016841F48041016070471E
:10108000000400580B490A6822F00702921C0A600B
:1010900009490A6842F004020A60012807D040BFEB
:1010A00020BF20BF086820F004000860704730BFF0
:1010B000F8E700000004005810ED00E00248006866
:1010C00000F4C06070470000000400580248016846
:1010D00041F4807101607047000400580F4A10B558
:1010E000002810680C464FEA80500ED0002801DB23
:1010F000FFF7C0FF0A48016821F004010160012CDC
:101100000AD040BF20BF20BF10BD0028F2DAFFF791
:101110008FFF0028F8D1EDE730BF10BD1404005850
:1011200010ED00E02DE9F047044600260068354642
:10113000B046C0034FF0B04740D5FFF7C7FFFFF7F9
:1011400003FF8146DFF878A105E0FFF7FDFEA0EB85
:10115000090002282AD8DAF80000C005F5D535BB09
:10116000D7F89000616B00F44070884211D0D7F836
:10117000900020F44076D7F8900040F48030C7F813
:101180009000D7F8900020F48030C7F89000C7F89E
:101190009060B0075FD5FFF7D7FE064641F2883969
:1011A00006E0FFF7D1FE811B494501D9032504E084
:1011B00001F033FD0128F4D1F5B3A8462078C0072B
:1011C00002D0606801F065FD2078800702D5A06834
:1011D00001F05FFD2078800607D52069D7F88810D8
:1011E00021F440610143C7F888102088800502D5AA
:1011F000206A01F043FD2088400502D5606A01F0B5
:101200003DFD2088000502D5A06A01F037FD207859
:10121000400602D5606901F022FD2078000602D563
:10122000A06901F01CFD2088C00502D5E06901F02D
:1012300016FD2078C00600E00DE019D5E068D7F86B
:10124000881021F440710143C7F88810E068B0F5B8
:10125000807F09D00CE0606BD7F8901021F44071CA
:101260000143C7F89010A9E7F86840F08070F86073
:10127000208800040DD5206BD7F8881021F040415C
:101280000143C7F88810206B18B9F86840F08070E7
:10129000F860208840040FD5E06AD7F8881021F064
:1012A00040510143C7F88810E06AB0F1005F03D1F4
:1012B000F86840F48030F8604046BDE8F0870000F0
:1012C000000400582DE9F0410D46040076D0DFF807
:1012D000B081D8F8000000F00700A84215D2D8F875
:1012E0000000474620F007002843C8F80000FFF739
:1012F0002BFE064604E0FFF727FE801B022874D869
:10130000386800F00700A842F5D120784FF0B046C9
:10131000800713D5A068B16821F0F0010143B160E6
:10132000FFF712FE074604E0FFF70EFEC01B02287F
:101330005BD8B068C0F300400028F5D020784006A4
:1013400017D56069D6F8081121F00F0141EA101095
:10135000C6F80801FFF7F8FD074604E0FFF7F4FDC3
:10136000C01B02287AD8D6F80801C0F30040002834
:10137000F4D02078400713D5E068B16821F4E0612B
:101380000143B160FFF7E0FD074604E0FFF7DCFD35
:10139000C01B022862D8B068C0F340400028F5D0D6
:1013A0002078000715D52069B16821F4605141EA21
:1013B000C001B160FFF7C8FD074605E02BE0FFF76D
:1013C000C3FDC01B022849D8B068C0F38040002884
:1013D000F5D02078C0072CD06068022806D00328FA
:1013E00007D0A8B101F00AFC05E037E001F000FCED
:1013F00001E001F02EFC70B16068B16821F00301DA
:101400000143B160FFF7A0FD064641F288370AE0CC
:1014100001F00AFCEFE70120BDE8F081FFF794FD41
:10142000801BB8421AD801F0DDFB6168B0EB810F78
:10143000F4D1D8F80000464600F00700A84214D9BD
:10144000306820F0070028433060FFF77DFD044638
:1014500006E0FFF779FD001B022801D90320DBE736
:10146000306800F00700A842F3D100F00FF80549FA
:10147000086005480068BDE8F041FFF785BD000041
:1014800000400058300000202800002010B500F077
:101490002FF84FF0B0418968044A01F0F00102EBE7
:1014A00091010968B0FBF1F010BD0000846F0008E5
:1014B00010B5FFF7EBFF4FF0B0418968072202EA51
:1014C0001121024A12F82110C84010BD0470000812
:1014D00010B5FFF7DBFF4FF0B0418968072202EA41
:1014E000D121024A12F82110C84010BD0470000832
:1014F0002DE9F0470024254601F074FB064601F073
:10150000A2FBDFF8C8804FF0B0474FEA480946B168
:101510000C2E04D0042E30D0082E2AD030E0012822
:101520002ED138682A49C0F3C00000283868C0F3BB
:10153000C00004D088B1386800F0F00011E018B1A4
:10154000386800F0F00003E0D7F8940000F4706011
:1015500000F4706001EB901007E0D7F8940000F4FD
:10156000706000F0F00001EB9000056846B92C4671
:1015700006E03868C0F3005008B1444600E04C462D
:1015800001F030FB0C281DD101F05DFB022805D0D5
:10159000032806D13868C0F3005008B1454600E082
:1015A0004D46F868F968C0F30620684301F0700200
:1015B000012101EB1212B0FBF2F2F86801EB50705E
:1015C000B2FBF0F42046BDE8F08700000024F400F0
:1015D000C46F00082DE9F041040077D001F002FB50
:1015E000064601F030FB074620784FF0B0458006F4
:1015F0007ED576B10C2E01D1012F0AD0206A0028A9
:10160000286864D040F001002860FFF79DFC804608
:101610004AE001F009FB10B1206A0028DDD0A16A80
:101620002868000703D5286800F0F00004E0D5F82A
:101630009400F02202EA1010814212D9084601F00B
:1016400081FE002842D1286840F008002860286800
:10165000A16A20F0F00008432860606A01F0EAFA0D
:1016600011E0286840F0080028602868A16A20F08E
:10167000F00008432860606A01F0DCFAA06A01F01B
:1016800061FE0028DED1FFF701FFF7490860F74847
:101690000068FFF779FC00287ED129E0FFF754FCB1
:1016A000A0EB0800022878D801F0BEFA0028F5D097
:1016B000286840F0080028602868A16A20F0F0003F
:1016C00008432860606A01F0B5FA11E0ABE020F051
:1016D00001002860FFF738FC804605E0FFF734FC86
:1016E000A0EB08000228DED801F09EFA0028F5D110
:1016F0002078C00748D0082E1ED00C2E01D1032F11
:101700001AD02868A16820F4801008432860606817
:10171000B0F5803F17D0B0F5041F286817D020F42B
:1017200080302860286820F4001028606068E8B1E4
:10173000FFF70AFC804614E001F05AFA20B3606813
:10174000002870D020E0286840F48030EDE740F4B5
:1017500000102860F7E7FFF7F7FBA0EB080064280C
:10176000A1D801F045FA0028F5D00DE0FFF7ECFB19
:10177000804605E0FFF7E8FBA0EB0800642892D85C
:1017800001F036FA0028F5D12078800737D5042EED
:1017900011D00C2E04D101E080E1D3E0022F0AD059
:1017A0002069002828681AD040F480702860FFF76C
:1017B000CBFB07460BE001F021FA60B1206900285D
:1017C000BFD008E0FFF7C0FBC01B02288BD801F098
:1017D00015FA0028F6D0606901F016FA0FE020F43F
:1017E00080702860FFF7B0FB074604E0FFF7ACFB12
:1017F000C01B0228B4D801F001FA0028F6D12078E5
:10180000000758D5A0690028D5F8940040D0E169B8
:1018100000F01002914225D081074FEAC07003D535
:1018200000288ED001E058E1A0B1D5F8940020F056
:101830000100C5F89400FFF787FB074604E0FFF7B7
:1018400083FBC01B11287DD8D5F89400C0F340005D
:101850000028F4D1D5F89400E16920F01000084385
:10186000C5F89400D5F8940040F00100C5F8940044
:10187000FFF76AFB074604E0FFF766FBC01B112871
:1018800060D8D5F89400C0F340000028F4D012E0EE
:1018900020F00100C5F89400FFF756FB074604E06E
:1018A000FFF752FBC01B11284CD8D5F89400C0F3A9
:1018B00040000028F4D1207840075FD5DFF8B081E0
:1018C000D8F80000C0F3002080B9FFF7FFFBFFF756
:1018D0003BFB074604E0FFF737FBC01B022831D86B
:1018E000D8F80000C0F300200028F4D0E06841F2EE
:1018F000883840B3852801D0052805D1D5F8900057
:1019000040F00400C5F89000FFF71EFB0746D5F82D
:10191000900040F00100C5F8900004E0FFF714FBD0
:10192000C11B41450ED8D5F89000C0F340000028F7
:10193000F4D0E06881280ED085280CD0FFF704FB96
:10194000074601E08EE024E0D5F8900020F080000A
:10195000C5F8900018E0FFF7F7FA0746D5F89000B1
:1019600040F08000C5F8900004E0FFF7EDFAC11BDD
:10197000414577D8D5F890000005F6D531E0FFF75E
:10198000E3FAC11B41456DD8D5F890000005F6D4A7
:1019900027E0FFF7D9FA0746D5F8900020F080003D
:1019A000C5F8900004E0FFF7CFFAC11B414574D899
:1019B000D5F890000005F6D4FFF7C6FA0746D5F82B
:1019C000900020F00100C5F8900004E0FFF7BCFA99
:1019D000C11B414561D8D5F89000C0F340000028F4
:1019E000F4D1E06AE8B30C2E5FD00228286820F01A
:1019F000807028600BD0E86820F00300E860E86899
:101A00001C490840E860FFF79FFA044648E0FFF7EA
:101A10009BFA064604E0FFF797FA801B0A283CD899
:101A200001F017F90028F6D1D4E90C010843D4E9F4
:101A30000E2141EA02210843216C0843616C0843EE
:101A4000E9680D4A11400843E860286840F080705A
:101A50002860E86840F08050E860FFF775FA0446B7
:101A600011E03CE019E000003000002028000020D8
:101A700000040058FFFFFEEE8C80C111FFF764FAEE
:101A8000001B0A2809D801F0E4F80028F6D026E067
:101A9000FFF75AFA001B0A2802D90320BDE8F0819B
:101AA00001F0D7F80028F3D119E00128F6D0E86852
:101AB000226B00F0030191420FD1626B00F07001C4
:101AC00091420AD1A26B00F4FE41B1EB022F04D186
:101AD000616C00F06040884201D00120DEE7002008
:101AE000DCE77047014850F82100704700B1004022
:101AF000014840F82120704700B1004010B590F82F
:101B00002C10012916D0012300F82C3F022141702E
:101B10000949CA220A6053220A60074A0C3A14682B
:101B200044F020041460FF220A6043700021017019
:101B3000084610BD022010BD2428004010B503F057
:101B4000C3FDBDE81040401C03F0D0BD10B50446F5
:101B500007480068400606D5054A40210832116052
:101B60002046FFF7EBFF012184F82D1010BD000087
:101B70005428004010B590F82C1001291BD00122E8
:101B800000F82C2F022141700C49CA230B6053230B
:101B90000B600A4B0C3B1C6844F080041C60084B33
:101BA0001C6844F480241C60FF230B6042700021F9
:101BB0000170084610BD022010BD0000242800401E
:101BC0008008005804F0BCBE2DE9F04105460C48E1
:101BD0000468286B0B4F0440E0074FF0010603D068
:101BE0003E602846FFF7EEFFA00704D502203860CC
:101BF0002846FFF776FF85F82D60BDE8F0810000EC
:101C0000542800405C28004070B590F82C20012A30
:101C100029D0012280F82C20022580F82D501A4C62
:101C2000CA23236053232360174B174E0C3B3836CF
:101C3000B1F5807F196818D021F408511960124954
:101C400028310B6823F000430B60016B21F0020187
:101C500001633560FF21216080F82D20002180F88C
:101C60002C10084670BD022070BD21F48851196007
:101C7000054920310B6823F000430B60016B21F014
:101C8000010101633260E5E72428004070B50400DB
:101C90004FF0010048D094F82D0028B9002084F8B6
:101CA0002C00204600F046F8022084F82D001F4E3C
:101CB000CA20306053203060204601F08FFB60BBAB
:101CC0001A4D0C3D28681A49084028602868616848
:101CD000A269084321691143084328602189E0680B
:101CE00040EA0140114914390860D4E90901084368
:101CF0000E4918390A6822F4F85210430860204649
:101D000001F092FB48B9D4E90721114362692B68BD
:101D100023F060431A4311432960FF2131600028FA
:101D200002D1012184F82D1070BD0000242800404C
:101D3000BFFF8FFB10B590B0044638216846FEF710
:101D4000B1FB18492068884229D180130090001205
:101D50000D906846FFF7E6F908B1FEF792FD4FF0E7
:101D6000B04050F8901F41F4004140F83819016824
:101D700041F4806101600068002200F480600E90F0
:101D800011460220FFF722F90220FFF711F9002285
:101D900011462A20FFF71AF92A20FFF709F910B097
:101DA00010BD0000002800402DE9F04F04460B460E
:101DB00094F82C100020012950D0012784F82C70B1
:101DC0004FF0020A84F82DA054490968534E01F4DB
:101DD00040754FF4807B0C3680465D451ED0E2B3E3
:101DE0005969B1F1803F07D0B1F5000F04D03068D8
:101DF000400601D483F8038098781A7893F803C0DA
:101E000040EA02405A78120242EA8C52104393F898
:101E1000242040EA02601A6A10430843DFF8FC906D
:101E2000CA2209F11809C9F800205322C9F8002074
:101E30009A6ADFF8E8C05A4532680CF1500C40D17C
:101E400022F488523260CCF80070344A38325D4552
:101E500026D1D3E90601084326E002E00220BDE8CE
:101E6000F08F3068400601D483F80380187801F0C1
:101E7000A9FA0204587801F0A5FA42EA00229878FB
:101E800001F0A0FA0243D87842EA805293F8240085
:101E900001F098FA196A42EA006008435969BCE700
:101EA0001E4934310860986910601C4958686431D3
:101EB0000860206B40F001002063306840F48850D7
:101EC0001CE022F408523260CCF800A0134A4032E1
:101ED0005D4503D1D3E90601084303E00F493C31D6
:101EE0000860986910600D49586868310860206B77
:101EF00040F002002063306840F408503060084829
:101F0000016841F400310160FF21C9F8001084F834
:101F10002D7084F82C800020A1E700000C280040E0
:101F20008008005870B50B4D286820F0200028600C
:101F3000FFF70AF804464FF47A7606E0FFF704F854
:101F4000001BB04201D9032070BD28688006F5D57A
:101F5000002070BD0C2800404FF0E020016941F0E6
:101F600002010161704700000448826819B101292B
:101F700003D1080210478020FCE77047340000209E
:101F80000149402089680847340000202DE9F041CC
:101F9000054680791F4616460C4601282CD16879E3
:101FA000012829D04FF0010885F80580284602F065
:101FB00037FC00F0FDFD2146284602F005FC00211B
:101FC000284602F001FC002406E03146284602F0D3
:101FD000CDFB641CA4B2761CBC42F6D300F0FAFD23
:101FE000284602F03FFCA86800B1012085F8068071
:101FF00000216971BDE8F0810220FBE72DE9F0477F
:1020000005468079984691460E46012831D1687977
:1020100001282ED001276F71284602F001FC4FF0F5
:10202000000A842E0BD0942E09D085F804A000F06D
:10203000BFFD3146284602F0C7FB002408E02F719F
:10204000F5E719F80410284602F0BEFB641CA4B2A0
:102050004445F6D300F0BEFD842E02D0284602F09F
:1020600001FCA86800B10120AF7185F805A0BDE8AA
:10207000F0870220FBE7000001492020896808471B
:1020800034000020014910208968084734000020EE
:1020900038B505460020009002236A4612212846E2
:1020A000FFF774FF9DF800009DF8011041EA002140
:1020B000CC43E00702D1284600F032F9A00702D451
:1020C000284600F019F9600702D4284600F092F87B
:1020D000200702D4284600F01DF9E00602D4284665
:1020E000FFF7D0FFA00602D42846FFF7C5FF600621
:1020F00002D42846FFF744FF200607D4E00501D4A8
:10210000012100E000212846FFF72EFFA00502D4A0
:10211000284600F0F7F802236A4619462846FFF7DA
:102120006DFF38BD2DE9F843040004D0A0790025E7
:102130002F4618B106E00120BDE8F88367712046FC
:1021400000F042F80220A0714FF0B040D0F8941097
:1021500021F40041C0F89410184964220968C1EBC9
:10216000C101C1F34C4111FB02F10126009100991C
:10217000C1B1491E0091D0F89410C1F380310029FB
:10218000F5D100F027FD0E48016841F4805101604F
:102190004FF40068404600F013FD0A49C1F8008082
:1021A0001DB107E00125A660EBE7206802F0CCFA3C
:1021B0002671A760A6712846BEE700003000002007
:1021C000900800581804005808B54FF0B040416E10
:1021D00041F001014166406E002200F001000090D4
:1021E00011463220FEF7F2FEBDE808403220FEF72D
:1021F000DFBE000001490420896808473400002040
:102200002DE9F041054680791F4616460C46012807
:1022100030D1687901282DD04FF0010885F805806C
:10222000284602F0FDFA00F0C3FC1E21284602F009
:10223000CBFA2146284602F0C7FA0021284602F0D0
:10224000C3FA002406E03146284602F08FFA641CE7
:10225000A4B2761CBC42F6D300F0BCFC284602F0C7
:1022600001FBA86800B1012085F806800021697192
:10227000BDE8F0810220FBE72DE9F04105468079B9
:102280001F4616460C46012834D16879012831D002
:102290004FF0010885F80580284602F0C1FA00F0E9
:1022A00087FC1D21284602F08FFA210A284602F0F9
:1022B0008BFAE1B2284602F087FA0021284602F0A4
:1022C00083FA002406E03146284602F04FFA641CE7
:1022D000A4B2761CBC42F6D300F07CFC284602F087
:1022E000C1FAA86800B1012085F806800021697153
:1022F000BDE8F0810220FBE7014902208968084718
:102300003400002002494FF400708968084700003B
:102310003400002001490820896808473400002063
:102320000149012089680847340000202DE9F04167
:10233000054680791E4617460C4601282BD1687940
:10234000012828D04FF0010885F80580284602F0C2
:1023500067FA00F02DFC0E21284602F035FA2146DE
:10236000284602F031FA002405E0395D284602F0E3
:102370002BFA641CA4B2B442F7D300F02BFC28461D
:1023800002F070FAA86800B1012085F806800021EB
:102390006971BDE8F0810220FBE72DE9F0410546B7
:1023A00080791E4617460C46012831D168790128EC
:1023B0002ED04FF0010885F805800220A87128462C
:1023C00002F02EFA00F0F4FB0D21284602F0FCF991
:1023D000210A284602F0F8F9E1B2284602F0F4F9A1
:1023E000002405E0395D284602F0EEF9641CA4B231
:1023F000B442F7D300F0EEFB284602F033FAA868A7
:1024000000B1012085F8068000216971BDE8F081E6
:102410000220FBE74FF0E020016921F00201016199
:10242000704710B5044690F8800001281CD00120A8
:1024300084F880002420C4F88400206801680268C1
:1024400022F00102026041F000504FF0005161663D
:1024500021680860204603F04DFB2020C4F884006A
:10246000002084F8800010BD022010BD90F880107C
:10247000012910D0012180F88010016851E8002F57
:1024800042F0020241E80023002BF6D1002180F83F
:10249000801008467047022070477047704770B53B
:1024A000044690F8800001281DD0012084F88000A7
:1024B0002420C4F8840020680568026822F0010224
:1024C00002602068826822F060620A4382602046CF
:1024D00003F010FB206805602020C4F88400002071
:1024E00084F8800070BD022070BD70B5044690F87D
:1024F000800001281DD0012084F880002420C4F829
:10250000840020680568026822F0010202602068E9
:10251000826822F060420A438260204603F0EAFAB1
:10252000206805602020C4F88400002084F8800022
:1025300070BD022070BD38B5044690F880000025BB
:10254000012812D0012084F880002420C4F88400DF
:102550002068036823F0010303602068836823F484
:1025600040130B43836011B10EE0022038BD206898
:10257000416893B221F01001194341602068120CA8
:10258000416862F31F6141602068016841F0010108
:102590000160FEF7D9FC03466FF07E4000900022F8
:1025A0004FF48001204603F0B7FF08B1032502E095
:1025B0002020C4F88400002084F88000284638BD1C
:1025C00070477047704700002DE9F04103680446EA
:1025D000D86919689A6840F60F0528424FF000053F
:1025E00009D186067ED501F0200602F080573E43D1
:1025F00078D0216F27E1A94EA94F16400F403743ED
:1026000070D0C70709D0CF0507D501271F62D4F8BE
:102610008C3043F00103C4F88C3083070AD5D3070C
:1026200008D0276802233B62D4F88C3043F00403BF
:10263000C4F88C3043070AD5D30708D02768042391
:102640003B62D4F88C3043F00203C4F88C300307AB
:102650000CD501F02003334308D0266808233362E9
:10266000D4F88C3043F00803C4F88C3003050BD544
:102670004B0109D526684FF400633362D4F88C30DF
:1026800043F02003C4F88C30D4F88C30002B3AD0BF
:10269000800609D501F0200002F08051084303D0E4
:1026A000216F09B120468847D4F88C0021688968D9
:1026B000490602D410F0280F27D0204603F028FB4B
:1026C0002068806840061BD52068083050E8001F4D
:1026D00021F0400140E80012002AF5D1E06F78B106
:1026E000704900E017E08163E06FFEF70EF9002803
:1026F00009D0E06F816B00E02046BDE8F04108475B
:102700002046FFF75FFFBDE8F0812046FFF75AFF44
:10271000C4F88C50F7E7E76E2026012F7ED1C7065C
:102720007CD5CF067AD510201862206880684006D4
:1027300042D5E16F086840680004000CE3D0B4F8AB
:102740005C208242DFD9A4F85E0008680068800639
:102750002BD4206850E8001F21F4807140E800125B
:10276000002AF6D12068083050E8001F21F001014E
:1027700040E80012002AF5D12068083050E8001F18
:1027800021F0400140E80012002AF5D1C4F8886029
:10279000E566206850E8001F21F0100140E80012B3
:1027A000002AF6D1E06FFEF779F8B4F85C00B4F8CF
:1027B0005E10401A81B22CE0B4F85C00B4F85E10F0
:1027C000401A81B2B4F85E0000289CD000299AD04B
:1027D000206850E8002F22F4907240E80023002B7C
:1027E000F6D12E4BDB432068083050E8002F1A400A
:1027F00040E80027002FF6D1C4F88860E566256719
:10280000206850E8002F22F0100240E80023002B3F
:10281000F6D12046FFF741FE75E7FFE7C70209D56D
:10282000570207D54FF4801018622046BDE8F041EA
:10283000FFF7C7BE03060AD501F0800302F40002C9
:10284000134304D0616F00297FF456AF5BE7420663
:1028500011D54A060FD52046016851E8002F22F015
:10286000400241E80023002BF6D1C0F884604567A0
:1028700000F066F947E7020206D54A0004D5204673
:10288000BDE8F041FFF79CBEC001C5D50029C3DA01
:102890002046BDE8F041FFF701BE00000100001036
:1028A00020010004615C000810B5040003D0D4F8D6
:1028B000840010B107E0012010BD002084F88000E2
:1028C000204600F043F82420C4F884002068016802
:1028D00021F001010160204603F06EFC0128EBD0DD
:1028E000A06A10B1204603F027F92068416821F45E
:1028F000904141602068816821F02A018160206850
:10290000016841F0010101602046BDE8104003F07C
:1029100077B9000010B5044600680B49884212D10F
:102920004FF0B040816D21F4003181650C214FF0F2
:102930009040FEF7A1F9A06FFEF720F8BDE8104027
:102940002520FEF724BB10BD0044004030B595B0F3
:10295000054614210EA8FDF7A5FD38216846FDF7B0
:10296000A1FD27492868884248D1264802240290C0
:1029700000946846FEF7D6FB08B1FDF782FF4FF0E2
:10298000B041886D40F400308865886D00F40030F7
:102990001390C86C40F00100C864C86C0EA900F028
:1029A000010013900C20CDE90E04012010900320AB
:1029B0001190072012904FF09040FEF707FA134C49
:1029C000114800212060142060601020C4E9020139
:1029D0008020C4E90401A161E16120462162FEF783
:1029E0008DF808B1FDF74DFFAC67002202212520CC
:1029F000A562FEF7EBFA2520FEF7DAFA15B030BD36
:102A00000044004004000C005800024084010020F3
:102A100030B4D0F88830202B20D1E1B1DAB190F871
:102A20008030012B1AD0012380F880300023C36648
:102A30000B4C0368A3420BD05B681B0208D50368EC
:102A400053E8004F44F0806443E80045002DF6D180
:102A500030BC03F0D5BC012030BC70470220FBE73E
:102A60000080004010B5044600680A49884210D131
:102A70000948836833B1D4F88C0018B900220121C9
:102A8000054898472046BDE8104001220249FFF75B
:102A9000BFBF10BD004400400C00002070B50446CC
:102AA000D0F88400202842D171B36AB394F8800032
:102AB00001283CD0012084F880002165A4F854202E
:102AC000A4F856200025C4F88C502120C4F88400B6
:102AD000A06FD8B11749C162A16F174813460863A8
:102AE000A16F16484863A06F85632668216D06F1C3
:102AF0002802A06FFEF766F840B11020C4F88C00E1
:102B000004F8805F20206060012070BD21684020B3
:102B1000086284F880502068083050E8001F41F0B7
:102B2000800140E80012002AF5D1002070BD02208B
:102B300070BD0000C55C0008075D0008755C0008FA
:102B400000680449884203D10349002049680847C6
:102B500070470000004400400C0000207047FEE772
:102B600008B54FF0B0418A6C02438A64896C014019
:102B7000009108BD08B54FF0B041CA6C0243CA6469
:102B8000C96C0140009108BD08B54FF0B041CA6C56
:102B90000243CA64C96C0140009108BD08B54FF0FA
:102BA000B041CA6C0243CA64C96C0140009108BDBF
:102BB0000248016821F40041016070479004005808
:102BC00003490A6822F4006202430A607047000069
:102BD000080400580248016841F400410160704750
:102BE000900400584FF0B040806800F00C0070472F
:102BF0004FF0B0400068C0F3404070474FF0B04025
:102C00000068C0F3802070474FF0B0414A6822F05E
:102C1000FE4242EA0060486070474FF0B040D0F892
:102C20009000C0F3400070474FF0B0400068C0F320
:102C3000400070474FF0B0414A6822F47F4242EAB8
:102C40000020486070474FF0B040C06800F00300BB
:102C500070474FF0B0400068C0F34060704710B557
:102C60004FF0B04353F8882F4FF47F2101EA10143E
:102C7000A24301EA001002431A6010BD4FF0B041B8
:102C800051F8882F030C1B049A4342EA0040086065
:102C900070474FF0B04151F8882F22EA104280B2BD
:102CA00002430A60704710B50420FFF759FF012066
:102CB000FFF756FF002202210F20FEF787F9BDE83B
:102CC00010400F20FEF774B930B585B01421684666
:102CD000FDF7E8FB0220FFF74DFF0120FFF74AFF59
:102CE0000420FFF747FF124D002238212846FEF747
:102CF00025F93820009001240021CDE901410391FC
:102D000069462846FEF762F84FF40410CDE900400A
:102D100069464FF090400294FEF758F800221146A1
:102D20000620FEF753F90620FEF742F905B030BD44
:102D30000004004830B58BB02C216846FDF7B2FB8B
:102D4000164815490024016004611F214461816017
:102D50004FF08041C0E906418D15C0E90845FEF7F6
:102D600095FF08B1FDF78DFD0C48FEF703FF08B194
:102D7000FDF787FD07944FF000500A950194CDE9C7
:102D80000540002269460548FFF70EF8002801D0EB
:102D9000FDF777FD0BB030BD00280040B0000020EB
:102DA000064910B5082008600846FFF7BBF900285F
:102DB00003D0BDE81040FDF764BD10BDE800002061
:102DC00010B502F013FCBDE8104002F0B9BA4FF0A4
:102DD000FF3003F0FFBC0000184810B51649016031
:102DE0004FF4E1314160002181600C22C160C0E9F3
:102DF00004128161C161016241628162FFF754FD89
:102E000008B1FDF73EFD00210C48FFF76EFB08B14D
:102E1000FDF737FD00210948FFF741FB08B1FDF739
:102E200030FD0648FFF7FDFA002803D0BDE810404A
:102E3000FDF727BD10BD000000440040F400002055
:102E4000FEE7FEE72DE9FC4116461C460D46074607
:102E5000012225A30021104603F0C6FBCDE9006442
:102E6000012224A30021104603F0BEFB20462A4C79
:102E7000FF21A070002020702848FDF713FBA580DB
:102E8000FF2D04D82A4639462448FDF7A4FA667077
:102E900023A3012200210320009503F0A5FB1F4D71
:102EA000244E00240022285D009023A31146032015
:102EB00003F09AFB04EA06000F2805D100220CA3B8
:102EC0001146032003F090FB641C202CEADB002257
:102ED00007A31146032003F087FBBDE8FC41002156
:102EE000012003F0E1BC00004F6E5278446F6E6524
:102EF0000A0D00005273736956616C75653D256457
:102F00002064426D2C20536E7256616C75653D25B0
:102F10006464420A0D000000180000200002002036
:102F20007061796C6F61642E2073697A653D2564E8
:102F3000200A0D000F0000802530325800000000EC
:102F400010B5012206A30021104603F04DFB0749EE
:102F5000022008700021BDE81040012003F0A4BC4D
:102F60004F6E52784572726F720A0D001800002081
:102F700010B5012206A30021104603F035FB0849D5
:102F800001200870BDE81040002103F08DBC000056
:102F90004F6E527854696D656F75740A0D000000AC
:102FA0001800002010B5012206A30021104603F0EE
:102FB0001BFB0749032008700021BDE810400120D9
:102FC00003F072BC4F6E5478446F6E650A0D0000BA
:102FD0001800002010B5012206A30021104603F0BE
:102FE00003FB0849042008700021BDE810400120BF
:102FF00003F05ABC4F6E547854696D656F75740A4E
:103000000D0000001800002010B5124C08212046C9
:10301000FDF78CFF10212046FDF788FF01220EA34B
:103020000021104603F0E0FA01220EA30021104611
:1030300003F0DAFA104811A10968C0F81B10114812
:103040002021826A0C481B309047BDE810400E4892
:1030500003F0E0BC000400482E2E2E504F4E470ACD
:103060000D000000536C6176652020547820737445
:103070006172740A0D000000E4020020504F4E47B8
:1030800000000000D470000800040020704710B554
:10309000FFF7C0F90121BDE810400020FEF71EB87F
:1030A00010B5FFF7B7F9034901200860BDE81040EB
:1030B000FDF7E8BF880400587047FEF74DBF10B514
:1030C000FEF74AFFBDE8104003F0E6BE704700007F
:1030D0002DE9F0474C4CE06A80474C4D4C4E40F691
:1030E000B839287805287DD2DFE800F003656563EC
:1030F0008100E878474F0028A8884FF001082FD0BA
:1031000000287FD04248042243A1E438FDF718F993
:1031100038B13F48042242A1E438FDF711F9C0B1AB
:103120001AE0414803F0B4FC002208213846FDF7BC
:1031300005FF10213846FDF7F9FEE06D8047C830E5
:10314000FDF788FD012239A30021104603F04CFA57
:103150003AE00020E8704AE085F8038036A347E0B3
:1031600000284FD02A4804222DA1E438FDF7E8F8C2
:103170000028F1D12C4803F08BFC002210213846A6
:10318000FDF7DCFE08213846FDF7D0FEE06D8047F4
:10319000C830FDF75FFD01222CA30021104603F08B
:1031A00023FA01222CA30021104603F01DFA1AA0D5
:1031B00011E02EA31CE0E878C8B1E06D8047A96853
:1031C0000844C830FDF746FD01222BA3002110461C
:1031D00003F00AFA12A020210068C6F81B000C4870
:1031E0001B3000E00EE0A26ABDE8F047104727A3BD
:1031F00001220021104603F0F7F94846616BBDE853
:10320000F0470847BDE8F087D47000081800002098
:10321000E402002000040048504F4E470000000028
:1032200050494E4700000000000400202E2E2E5072
:10323000494E470A0D0000004D61737465722052BB
:10324000782073746172740A0D0000002E2E2E50C7
:103250004F4E470A0D000000536C617665202054E4
:10326000782073746172740A0D0000005278207324
:10327000746172740A0D00004D617374657220549C
:10328000782073746172740A0D000000536C6176CB
:10329000652052782073746172740A0D000000007A
:1032A000FDF720BAFDF740BAFDF743BAFDF743BA80
:1032B000FDF76FBAFDF76FBA70B5204A88B0F2E833
:1032C0000234CDE90334F2E80234CDE905341CCAF6
:1032D0008DE81C000024B1F5007F6A46214607D026
:1032E00005AB33F8115085420BD352F821400BE067
:1032F00003AB33F811508542F7D2491C0329F8D3A8
:1033000002E0491C0329ECD30D4E306820F0070081
:1033100020433060FDF718FE054607E0FDF714FE78
:10332000401B022802D9032008B070BD306800F0AD
:103330000700A042F2D10020F6E70000406F00082D
:10334000004000583C2101EA90000C4910B5085893
:103350004FF0B041D1F80811094A01F00F0152F8BD
:103360002110B0FBF1F4FDF7A9FE01460548B4FBBE
:10337000F0F0BDE81040FFF79FBF0000C46F0008E9
:10338000846F000840420F00704770474FF0FF30D5
:10339000704700207047002070474FF0FF307047A3
:1033A0004FF0FF3070477047704770474FF0FF3065
:1033B00070474FF0FF3070470148FEF705BC000032
:1033C000B0000020002102E00A38C0B2491C0A28DF
:1033D000FAD2090740EA1160704700002DE9F04772
:1033E000104F064600243868400618D4386840F06C
:1033F00080003860FDF7A8FD05464FF47A794FF05C
:10340000030807E0FDF7A0FD401B484502D903244F
:1034100086F82D803868400601D4032CF2D120466E
:10342000BDE8F0870C2800402DE9F041054613481F
:103430000024016821F080010160104E0C363068D4
:103440004FF00307800607D42846FEF76BFD90B1C6
:1034500085F82D7003240EE0306820F020003060E5
:103460002846FEF75FFD10B185F82D700324306803
:1034700040F0200030602046BDE8F0810C2800407C
:1034800001207047F0B50025DDE90564121D079F96
:10349000052901D0062902D10C2B00D20C2310B132
:1034A000012802D004E00B2901D00C2900D101250C
:1034B0000FB1102000E0002000EBC4004C4200EBF4
:1034C00084040EB1002000E0142020448C00062962
:1034D00002D9083005B1083C002800DA0020204459
:1034E000401E90FBF4F00C3300FB0230062900D89C
:1034F000801C012202EB8000891E8840F0BD10B5BF
:1035000001F080FA042805D0052805D0072805D049
:10351000002010BD022010BD012010BD032010BDF1
:1035200010B501F0C6FAC01C10BD000038B51E4928
:103530001E4D002448606C706C60AC601C48AC652B
:1035400001F012FB6C732C7301F0FDFC00210846A6
:1035500001F07DFB04220021012001F011FE002377
:103560004FF6FF701A46014601F0B0FB01F010F86B
:1035700000220E48551E0F4B29465C30009403F084
:10358000A7F90A480C4B002229467430009403F036
:103590009FF906485C3003F07BFABDE838400348E9
:1035A000743003F075BA00004000002018050020B8
:1035B0000139000829390008113900082DE9FC41BA
:1035C0000026954D8DF800600196B5F85400934C97
:1035D00020287CD015DC40F60217042878D00ADCBD
:1035E000012832D0022844D105F1740003F050FACA
:1035F0006878E0B350E008286BD0102839D188A350
:10360000F3E0402866D080287ED0B0F5807F71D06E
:10361000B0F5007F2DD185A301220021022002F008
:10362000E3FF01F0EFF9042879D001F0EBF9052868
:103630001FD17948743003F02BFA002001F038FDD7
:103640006068002815D0C06881E073485C3003F0E2
:103650001FFA002001F02CFDFFF79DFE012801D18B
:10366000FFF793FE6068002803D000686FE002E077
:103670008047BDE8FC81002001F01AFD002138469A
:1036800001F042FE40F64416304601F0BBFA40F02D
:103690000201304601F038FEFF226946684801F019
:1036A000F1F95D48243001F0B3F960680028E0D0FA
:1036B0008668002EDDD095F8240001281BD001A9D2
:1036C000E86B01F051F94FF47A71019804E07BE066
:1036D00040E06CE08FE017E000F5FA7090FBF1F04D
:1036E00043B2606895F929209DF800108468544819
:1036F000A047BEE714E095F9313095F930209DF8E8
:1037000000104F48B047B4E7002001F0D1FC6068DA
:103710000028AED081690029ABD000200AE00BE080
:10372000002001F0C5FC60680028A2D08169002952
:103730009FD0012088479CE737485C3003F0A8F908
:10374000002001F0B5FC6068002892D04068002895
:103750008ED18EE73BA301220021022002F044FF1C
:10376000A86D002885D0C0F3074140F6031000F093
:10377000B9FF35F8580FC0F3072140F6041000F0E8
:10378000B1FF297840F6051000F0ACFF384600F094
:10379000E2F840F00101384600F0A4FF002340F2B7
:1037A00062201A4601462E6001F090FA61E728A3D4
:1037B00001220021022002F017FFFFF7EAFD012895
:1037C00097D1FFF7F0FD54E71348743003F060F928
:1037D000687810B9002001F06BFC6068002888D080
:1037E000C068002885D080471CA301220021022048
:1037F00002F0FAFE3DE71CA301220021022002F0A4
:10380000F3FE687810B9002001F052FC60680028CF
:1038100091D000699BE700001805002040000020BF
:10382000484452204F4B0D0A000000004952515F9E
:1038300052585F54585F54494D454F55540D0A0036
:1038400018040020505245204F4B0D0A0000000084
:1038500053594E43204F4B0D0A000000484452205C
:103860004B4F0D0A000000004952515F4352435F25
:103870004552524F520D0A002DE9F04180468AB060
:103880001D4616460F460124002001F011FC0020C1
:1038900000F090F9404601F065FB00200121CDE9E0
:1038A0000801079006900290039004900590032071
:1038B000CDE9007000234FF416723946184600F027
:1038C000BBF9002000F04EF801F0F3F8C01CFDF742
:1038D000C1F903F01BF8074605E001F01BF9B042FF
:1038E00001DD002404E0384603F01AF8A842F4D3BE
:1038F000002001F0DDFB0AB02046BDE8F0810000A9
:103900000249A1F85400FFF759BE00001805002035
:1039100004484068002803D0C068002800D0004751
:10392000704700004000002004484068002803D091
:103930004068002800D00047704700004000002089
:10394000002310B51A461946184601F0BFF9BDE824
:10395000104001F0B0B801F055B901F05FB901F0C5
:10396000D9B8000010B50446FFF713FD012820D098
:10397000002340F262201A46014601F0A7F934B153
:1039800021460F4803F02AF80D4803F043F80C4C89
:103990000020743C0021A06594F8560001F0A1FBC2
:1039A0006078012808D0A0688001BDE8104001F0CF
:1039B00015BBFFF7F2FCE2E76FF07F40F5E7000090
:1039C0008C05002010B50446FFF7E3FC012820D049
:1039D000002340F262201A46014601F077F934B123
:1039E00021460F4802F0FAFF0D4803F013F80C4C83
:1039F0000020743C0021A06594F8560001F071FB92
:103A00006078012808D0A0688001BDE8104001F06E
:103A1000F9BAFFF7C2FCE2E76FF07F40F5E700007C
:103A20008C0500202DE9F84380460C46002340F227
:103A300001201A46014601F049F9484D012195F847
:103A4000560001F04EFB287840F68906012803D184
:103A500095F85100062812D0304601F0D3F840F016
:103A60000401304601F050FC3C4F28780E37022606
:103A700005282CD2DFE800F00B090B363E0030465B
:103A800001F0C0F820F00401EBE7EC772CE0FFF741
:103A900080FC012801D0AC7526E06A4621464046EC
:103AA000FFF784FC38B12EA301220021022002F08E
:103AB0009BFDBDE8F8839DF80000A875384601F02D
:103AC000BDF99DF800100022404601F0B7F82348E8
:103AD00069685C3002F082FFBDE8F8431F485C3043
:103AE00002F098BFAE73AC76384601F0A7F9002219
:103AF0002146E9E7224641461F4803F092F8B046C6
:103B0000AE73661CAE76384601F098F90021F120BC
:103B100000F0E8FD0021F02000F0E4FDA86C64282E
:103B200016D0E121F32000F0DDFD0421F22000F0A9
:103B3000D9FD08EBC404210AF42000F0D3FDE1B262
:103B4000F52000F0CFFDF1B26FF07F420A48BCE7EC
:103B50007021F32000F0C6FD1D21E7E718050020C5
:103B6000526164696F53656E64204F766572736944
:103B70007A650D0A000000001804002001F0F2B977
:103B800030B404460A4A094B02F10E00012C07D05A
:103B9000547D012C07D11970917530BC01F04EB9DC
:103BA0001970D177F9E730BC704700004000002061
:103BB0001805002070B5114C06462070FFF7F5FB84
:103BC0000025062E04D2DFE806F0050703131305CF
:103BD00003200EE000200CE0012001F09BF9617B46
:103BE000207B814208D06073BDE8704000F008B8C7
:103BF000022001F08FF9657370BD000018050020E8
:103C000070B504460B48047344730120FFF7D2FFDC
:103C10004FF4E860451C24B1342101F075FB4421C8
:103C200003E0142101F070FB24212846BDE8704018
:103C300001F06ABB180500202DE9FF4F87B0DFF8BF
:103C40008CB2DDE91565DDF87480179F14468A464D
:103C50008BF80180FFF798FBB8F1000F00D000252A
:103C6000DFF86C921FB1189889F8000002E0FF217C
:103C700089F800104FF6FF7101EAC60893490798CA
:103C800001F138020E31CDE9001200286CD0012874
:103C90007ED005287DD1012001F01CFA00278BF889
:103CA00038700920CBF83C408BF844004FF4487042
:103CB000CBF840005E46504600F090FE86F8450086
:103CC000B773A6F81080B7741020F0743775777545
:103CD00099F80000B0750120F07537760520FFF7E0
:103CE00069FF019801F028F8009801F0A7F879A081
:103CF000D0E90010CDE9021002A801F006FA40F266
:103D0000FF1001F0C5FA40F6B8073846FFF723FE6A
:103D100020F01001384600F0E5FC0421781C00F08A
:103D2000E1FC40F69B073846FFF715FE20F01C002B
:103D300040F00801384600F0D5FC40F2D167384623
:103D4000FFF709FE40F01801384600F0CBFC40F2C6
:103D5000AC673846FFF7FFFD20F0700040F05001DF
:103D6000384600F0BFFC43E0002001F0B3F900202A
:103D70008BF838000B20CBF83C408BF844005E46B3
:103D8000504600F02BFE86F845000020B07301E09D
:103D900037E033E0A6F810800420B0741820F074E7
:103DA0000020307587F00100707599F80000B0753B
:103DB000199808B1F22000E00120F075012030765A
:103DC000002001F075F90020FFF7F4FE019800F0E3
:103DD000B3FF009801F032F840A0D0E90010CDE91F
:103DE000041004A801F091F940F2FF1001F050FA1C
:103DF0004FF4FA504543B5FBF4F0B0600BB0BDE8AA
:103E0000F08F002001F066F90121364B8BF8381055
:103E1000E0B28BF8500013F80A208BF851200A9A70
:103E2000D8468BF85220BAF1000F03D0BAF1010F37
:103E300002D003E00B2C0BD00C2C09D0002288F808
:103E4000532088F80E10052805D0062803D008E076
:103E500088F85310F5E70C2E03D20C20A8F81C00AC
:103E600001E0A8F81C6088F81E7099F8000088F836
:103E70001F00199888F820001C9888F8210000205D
:103E800001F016F90120FFF795FE019800F054FFAC
:103E9000009800F0D3FFE8B200F033FF98F821005B
:103EA00040F23674012820460BD000F0ABFE40F003
:103EB0000401204601F028FA4FF6FF70C8F8080008
:103EC0009CE700F09FFE20F00401F2E718050020B7
:103ED00040000020B227000000000000C194C10093
:103EE000000000005871000870B50C4E054601EB4B
:103EF0004500B0650C4600234FF6FF701A46014698
:103F000000F0E4FE96F85600002101F0EAF82146A0
:103F10002846BDE8704001F08FB800001805002069
:103F20002DE9F04F814689B000201E4615460C460B
:103F30000746079000900190FFF726FA15B100267A
:103F4000012000E00020DFF8F8814FF0FF3B414600
:103F500088F8010001F1380201F10E01CDE90512E6
:103F60005FEA09004FF6FF7A4FF0010902D00128FD
:103F700060D17DE0A068002879D0E068002876D084
:103F8000A27F082A73D86846216902F0FFFB2068E7
:103F900000B1012001F09EF888F83870A068C8F8D8
:103FA0003C0094F8200088F84400454654F8040F7B
:103FB00000F014FD85F84500AF7321890AEAC100BD
:103FC0002882E07EA874A07EC000E874607F287517
:103FD000A07F241F78B3FF21A97594F8240002283C
:103FE0002DD094F82200022829D094F82300E875F7
:103FF00094F82400287694F822006875002001F0D7
:1040000057F80020FFF7D6FD069800F095FE0598BA
:1040100000F014FF684601F078F8A08B01F038F941
:10402000208B00F02BFE4FF4FA504643A068B6FBFD
:10403000F0F0A86079E0FFE7207DA875CDE794F85F
:104040002300F12803D0F22801D0012837D13D48C0
:104050008DF810703A4A03944168743202A8FFF751
:1040600095F920B92F7685F817906F75C6E726E089
:10407000208E20B394F83200012824D0FF25A06AB6
:1040800000B1012001F026F8F0B200F03AFE88F805
:10409000389094F82C0088F8500094F82D0088F897
:1040A000510094F82E0088F8520094F82F004946E9
:1040B000464680B101283AD002280ED105E0584684
:1040C00009B0BDE8F08F257DD9E794F82C000B28C6
:1040D0002DD00C282BD086F8537006F80E1F34F81C
:1040E000300FF081A078307475742079B0746079E5
:1040F000F074002000F0DCFF0120FFF75BFD069864
:1041000000F01AFE059800F099FEF07C0E3E40F299
:104110003674012820460DD000F074FD40F00401F3
:10412000204601F0F1F8C6F808A00798C8E786F81D
:104130005310D2E700F066FD20F00401F0E7000024
:1041400018050020400000202DE9FF4F85B01F46D4
:10415000DDE9145B8046DDF858A0129CFFF714F9E6
:10416000544E002206F1380000902A384FF0010921
:104170000390B8F1000F06D0B8F1010F44D0B8F1A8
:10418000040F40D17DE086F838200B20F46386F8D8
:1041900044009046384600F021FC86F84500079818
:1041A00030644FF6FF7086F80E8000EAC50030825A
:1041B0000420B0741820F07486F814808BF001008D
:1041C0007075BAF1000F02D0F220F07501E086F8A8
:1041D000179086F81890002000F06AFF0020FFF783
:1041E000E9FC009800F0A8FD039800F027FE32A03B
:1041F000D0E90010CDE9011001A800F086FF40F2DF
:10420000FF1001F045F849E02D4B86F83890E0B2F8
:1042100086F85000DB5D86F85130139B494686F8DE
:10422000523017B1012F02D003E00B2C09D00C2C17
:1042300007D086F85320B173052805D0062803D08F
:1042400007E086F85310F6E70C2D02D20C20B0835D
:1042500000E0B5831B4886F81EB00078F07786F83A
:1042600020A0199886F82100002000F021FF0120ED
:10427000FFF7A0FC009800F05FFD039800F0DEFD62
:104280000CE00420FFF796FC022086F83800162088
:10429000B46486F84C00009800F04EFD069800F0DB
:1042A00087FE86F85600FFF77FF81A98706009B00D
:1042B000BDE8F08F18050020C194C1000000000087
:1042C000587100084000002070B50D4601464FF4BB
:1042D0007A7002FB00F4084600F044FE284600F025
:1042E00067FE012100F0FDFE00F040FF214604487A
:1042F00002F074FBBDE87040014802F08BBB000087
:10430000740500202DE9FF4F87B000260C4680463B
:1043100000960196FFF738F89C4DDFF86CB205F176
:10432000380002902A3801274FF6FF794FF0040A2F
:104330000390B8F1000F61D0B8F1010F7ED0B8F151
:10434000020F7CD0B8F1030F7AD1A27C082A78D86A
:104350006846A16802F01AFA2068002871D042F27B
:10436000107188420BD80320A87385F838002068A4
:10437000E863E07C4FF0020885F844000CE0AE737F
:1043800085F838602068E863E07C85F844002068A0
:104390004FF0000880082864A18809EAC10028823B
:1043A00085F812A0A07CC000E8742E75A07D0228BC
:1043B0000DD0207D02280AD0607DE875A07D28768A
:1043C000207D6875002000F073FE404649E0607D66
:1043D000F12803D0F22801D0012832D16B4A04948D
:1043E0008DF818705C3204A8DBF80410FEF7CEFFDD
:1043F000002826D12E76EF756E75E3E72068002839
:104400001FD0A27C082A1CD86846A16802F0BEF919
:1044100085F838602068E863E07C85F84400A0698E
:104420002864AE73A18809EAC100288285F812A029
:10443000A07CC000E8742E75A07D03E039E080E028
:1044400097E071E002281ED0207D02281BD0607DFD
:10445000E875A07D2876207D6875002000F028FE94
:104460000020FFF7A7FB029800F066FC039800F01D
:10447000E5FC684600F049FE208A00F009FFA089AB
:1044800000F0FCFB75E0607DF12803D0F22801D03C
:1044900001285BD13D4A8DF8187004945C3204A861
:1044A000DBF80410FEF772FFF0BB2E76EF756E7529
:1044B000D3E785F83870207885F85000607885F863
:1044C0005100A07885F85200E07840B1012830D042
:1044D000022806D120780B282BD00C2829D085F86B
:1044E0005360AF73A088A883A079A877E07985F896
:1044F0002000207A85F82100002000F0D9FD01205D
:10450000FFF758FB029800F017FC039800F096FCA8
:1045100095F8510040F68904062820460CD000F09A
:1045200071FB40F0040100E010E0204600F0ECFEDA
:104530001FE085F85370D4E700F064FB20F004011D
:10454000F1E7206810B1B0F57A7F04D94FF0FF3061
:104550000BB0BDE8F08F0320FFF72CFB022085F89D
:1045600038002068A864162085F84C00029800F0F6
:10457000E3FB099800F01CFD85F85600FEF714FFD8
:104580000A9868600020E3E740000020180500203A
:1045900010B5042000F06CFDBDE810400220FCF7CF
:1045A00059BB002000F084BD084810B590F85600B3
:1045B000002100F096FD00234FF4C0701A4601461A
:1045C00000F084FBBDE8104000F04CBB1805002053
:1045D000FEB51F4616460D46DDE90A23DDE908CE85
:1045E00001004FF000004FF0010402D0012949D131
:1045F00014E0BEF1000F05D0002000EBCC011BB190
:10460000022002E00820F8E70020104401EBC0007F
:104610004FF47A7118304843344633E0CDF800E067
:10462000CDE9012363463A4631462846FEF72AFF84
:104630004FF47A71484316490024495D0B2921D271
:10464000DFE801F0060C12181B1D1F20090F1500D2
:1046500041F6846416E042F6B10413E043F60954CF
:1046600010E045F261140DE047F612240AE04AF228
:10467000C32407E04FF2244404E0064C02E0064C59
:1046800000E0064C2044401EB0FBF4F0FEBD0000EC
:104690005871000848E8010090D0030020A10700ED
:1046A00010B500F085FC012100F01BFDBDE81040B5
:1046B00000F05CBD094810B590F85600012100F0EB
:1046C00010FD2D214FF4D76000F00CF800F053FDE1
:1046D000BDE81040024800F035BD0000180500207C
:1046E000FFFF0F0000F010BE00F018BE70B50546C9
:1046F000FEF7DEFD01280CD140F62314204600F021
:1047000081FA20F0060129432046BDE8704000F000
:10471000FBBD70BD0021020C01D110210004020E6E
:1047200001D100020831020F01D10001091D054A23
:1047300002EB107000780844C0B2C0F11F00C0B294
:10474000704700005B71000807490A6822F04002C8
:104750000A6040F4417008604FF4B850486008683F
:1047600040F04000086070470000015878B5144AD6
:104770000446002012686423C2EBC202C2F34C421A
:1047800012FB03F60F4A01250096009B8BB15B1EBE
:10479000009393689B07F8D5FF2313730096009B43
:1047A00053B15B1E00939368DB07F8D0D2680A70A0
:1047B00078BD0120A560EFE70120A560F6E70000C5
:1047C000300000200000015878B5134A044600204C
:1047D00012686423C2EBC202C2F34C4212FB03F61E
:1047E0000E4A01250096009B7BB15B1E00939368E7
:1047F0009B07F8D511730096009949B1491E0091A5
:104800009168C907F8D0D16878BD0120A560F1E7AB
:104810000120A560F7E700003000002000000158EB
:1048200038B50446007901280ED10A48006800EB2B
:104830004000C0F34F300090FEF7BAF90099491ECE
:104840000091FCD1FEF7C6F92046BDE8384000F0E3
:1048500009B80000300000200148FDF719BC000035
:10486000E800002018B50F490446002009686422BA
:1048700001EB4101C1F34B4111FB02F10A4A0091E6
:104880001168009BC1F380013BB15B1E009313686C
:10489000C3F340030B42F3D118BD01200221A160F4
:1048A00018BD00003000002014040058C0F380112F
:1048B0008901C0F3401241EA4211C0F3001241EAFB
:1048C0000211C0F3C00241EAC201C0F3800241EA12
:1048D0008201C0F3400241EA420108B500F0010044
:1048E00001438DF8001001226946892000F0FCFC8C
:1048F00008BD0000174908B5884204D9E1208DF8A9
:104900000000E9201EE01449884204D9D7208DF820
:104910000000DB2016E01149884204D9C1208DF83F
:104920000000C5200EE00E49884204D975208DF89C
:104930000000812006E00B49884205D96B208DF8E4
:1049400000006F208DF8010002226946982000F0D7
:10495000CBFC08BD00E9A43580F8A9328044E52DE0
:10496000000B6B1B40FC5419F8B5064618A00D4609
:104970000068009040F6070000F044F9C0F3C1025F
:1049800000F007001DF80210401E81401148B0FBE6
:10499000F1F4B4FBF6F10120082900D202204143D2
:1049A000042900D2042044434FF4D66000F02AF9D1
:1049B0000007060D40F2B16000F024F93043010514
:1049C00001D50549084361094143C8112860F8BD74
:1049D00004080A0C0048E80100F0FFFF48B1084A4B
:1049E000002152F83130834205D902EBC100007931
:1049F00070471F207047491CC9B21629F1D3FEE742
:104A000024700008014840787047000034000020FE
:104A100038B5044603226946142000F0E3F818492B
:104A20008878207048B1012817D014220021204630
:104A300001F0B5FE0F20207038BD9DF800002071F8
:104A40009DF8010040424010A0719DF802004042D4
:104A5000401060710020A06038BD9DF80000404209
:104A6000401020739DF90100801C801060739DF838
:104A7000020040424010A0734868206138BD000029
:104A800034000020F8B505460E4600208DF80000E1
:104A900014466946304600F049F83278A24201D9FE
:104AA0000120F8BD29469DF8000000F08BF8002099
:104AB000F8BD01207047F8B5002040F6E2060090EE
:104AC000304600F09FF8054620F00101304600F026
:104AD0001BFCF71C384600F095F8044620F08001D6
:104AE000384600F011FC6FF07F4000F077FA0422A6
:104AF000694640F6190000F091F8002000F0D8FA5D
:104B00002946304600F000FC2146384600F0FCFB08
:104B10000098F8BD08B501226946152000F062F83A
:104B20009DF80000404240F3470008BD38B50D46EF
:104B3000044602226946132000F054F8094881789F
:104B4000012902D1C078012806D09DF8000020700C
:104B50009DF80100287038BD40F2027000F052F854
:104B6000F5E700003400002070B5154C00B1A060DE
:104B7000FEF716F90220FFF7B9FD0020207000F0C3
:104B800097FAFEF797FB40F6111501280CD020216B
:104B9000284600F0B9FB2021681C00F0B5FBFEF7A9
:104BA00085FB0120607070BD4021012000F0B6FA45
:104BB0000021284600F0A8FB7F20FFF777FEEEE7F4
:104BC0003400002010B5EFF3108472B613460A4685
:104BD00001460348FDF714FB84F3108810BD000064
:104BE000E800002010B5EFF3108472B613460A46B1
:104BF00001460348FDF7CAF984F3108810BD000090
:104C0000E800002008B5014601236A460248FDF786
:104C100033FB9DF8000008BDE800002010B5EFF35D
:104C2000108472B613460A4601460348FDF724FB7A
:104C300084F3108810BD0000E800002010B5144671
:104C400000F07CF92046BDE8104000F07BBA08B5C2
:104C500002228DF800008DF8011069468F2000F0C7
:104C600043FB08BD10B500221146C52000F03CFBF7
:104C700001490720487010BD3400002008B5010A22
:104C80008DF800108DF8010005488078002805D1C6
:104C90000222694640F2BE6000F040FB08BD000001
:104CA0003400002008B5010A8DF800108DF80100CD
:104CB00005488078002805D10222694640F2BC6090
:104CC00000F02CFB08BD0000340000201CB5040AD5
:104CD0008DF800408DF80100080A8DF80200100AD6
:104CE0008DF804008DF80520180A8DF806008DF85F
:104CF000031008228DF807306946104600F0F4FAD8
:104D00001CBD01B501226946A02000F0EDFA9DF816
:104D1000000040280ED34008002102E08008491C12
:104D2000C9B21F28FAD801EBC000C1B240F2067028
:104D300000F0EAFA08BD00007CB5044600203449C2
:104D40000090019020788978884201D000F0E2F844
:104D500020783049E0B101284BD002283BD003280D
:104D600015D160680522B1FBF0F0010C8DF8001040
:104D7000010A8DF801108DF80200207B8DF80300E8
:104D8000607B8DF8040069468B2000F0ADFA7CBD95
:104D900060680825B1FBF0F0010C8DF80010010AE5
:104DA0008DF801108DF80200207B8DF80300607BE8
:104DB0008DF80400A068184AC10940060023FBF7DB
:104DC00029FA010C8DF80510010A8DF806108DF8EE
:104DD00007002A46D7E720690422B1FBF0F0010C56
:104DE0008DF80010010A8DF801108DF80200207D69
:104DF0000AE0207E8DF80000607E8DF80100A07E24
:104E00008DF80200E07E04228DF80300BBE700006D
:104E1000340000200000093D0048E80108B58DF885
:104E200000008DF801108DF802208DF80330042267
:104E30006946952000F058FA08BD00003EB50446CA
:104E40000020334D0090019002902078A97888428C
:104E500001D000F05FF8207828B101283ED0022868
:104E600037D0032852D1607AF12802D0F2280AD034
:104E700012E04FF6FF70FFF715FF48F20500FFF74D
:104E8000FDFE022008E041F60F50FFF70BFF41F254
:104E90002100FFF7F3FE062061880922090A8DF838
:104EA0000010A1788DF8011021798DF80210617938
:104EB0008DF80310A1798DF80410E1798DF80510B3
:104EC000217A8DF806108DF80700A07A8DF8080079
:104ED00018E0207B01228DF8000013E0E089062213
:104EE000010A8DF800108DF80100207CE8708DF823
:104EF0000200607C8DF80300A07C8DF80400E07C4B
:104F00008DF8050069468C2000F0EEF93EBD0000EA
:104F10003400002001B508499DF80000887020B9D0
:104F2000002140F2AC6000F0EFF9012269468A20CE
:104F300000F0DAF908BD0000340000200A460146FE
:104F4000002000F0C1B908B5FEF7B2F9012800D081
:104F500000208DF8000001226946962000F0C4F977
:104F600008BD000038B5104D0446287820B9204609
:104F7000FFF7C0FC01212970E10960060B4A0023FC
:104F8000FBF748F9010E8DF80010010C8DF80110A7
:104F9000010A8DF802108DF803000422694686206C
:104FA00000F0A2F938BD0000340000200048E801FC
:104FB00070B505460124FEF777F920B1012805D028
:104FC000022803D101E00F2D00DD02240222294630
:104FD000204600F0D5F8204670BD0000084A08B50C
:104FE00005215170010C8DF80010010A8DF8011097
:104FF0008DF8020003226946822000F075F908BD91
:105000003400002038B50B4904460520487097212C
:1050100040F6AC0000F078F9200C8DF80000200A72
:105020008DF801008DF8024003226946822000F0CD
:105030005BF938BD340000201CB5020C8DF800204F
:10504000020A8DF801208DF80200080C8DF803008B
:10505000080A8DF804008DF8051006226946942090
:1050600000F042F90149062048701CBD34000020C0
:1050700038B504460020FEF713F90220FFF736FB8F
:10508000C4F380008000C4F3400140EA410004F012
:10509000010108438DF8000001226946842000F0D8
:1050A00023F902490020487038BD00003400002078
:1050B00001B501226946802000F016F99DF8001024
:1050C000034811B10221417008BD0121FBE7000036
:1050D0003400002001B5012269469F2000F004F948
:1050E00008BD10B5012401290AD1012802D00228E7
:1050F00005D005E002240420FFF7F8FA00E00324BD
:105100002046BDE81040FEF7CBB810B50146082296
:105110004FF4D86000F002F9002010BD08B500F08F
:1051200007008DF80000080C8DF80100080A8DF8C2
:1051300002008DF8031004226946972000F0D4F88D
:1051400008BD0000084A08B504215170010C8DF813
:105150000010010A8DF801108DF802000322694643
:10516000832000F0C1F808BD340000200022114661
:10517000D12000F0B9B800221146D22000F0B4B816
:10518000F8B515460C4640F6E706012820D040F653
:10519000D8073846FFF736FD40F01E01384600F0CC
:1051A000B3F80120FEF77EF80746BC4200DD7CB272
:1051B000142F3CD0112F43D00E2F4FF001034FF08E
:1051C000000248D007210420FFF728FE381B3FE0EB
:1051D0000020FEF767F80746BC4200DD7CB20E2FC8
:1051E00014D04FF001030A2F1A464FF0000116D0D9
:1051F0000620FFF713FE381BC0F10E0044B26FF01B
:105200001000844200DA0446182133E001231A46D4
:1052100000210420FFF702FEC4F10E00ECE701209C
:10522000FFF7FCFDC4F10A00C0F10D00E6E7012321
:10523000002205210320FFF7F1FDC4F1140007E06F
:105240000123002203210220FFF7E8FDC4F1110031
:10525000C0F1160007E002210846FFF7DFFDC4F1A8
:105260000E00C0F10E0044B26FF00800844200DA74
:1052700004463821304600F047F88DF800408DF89C
:105280000150022269468E2000F02EF8F8BD000081
:1052900070B504460B488078002812D14FF4D765CA
:1052A0002846FFF7AFFC00F0FE00C4F300210143E5
:1052B000284600F029F8E1B2681CBDE8704000F013
:1052C00023B870BD3400002010B5EFF3108472B61F
:1052D00013460A4601460348FDF728F884F3108870
:1052E00010BD0000E800002010B5EFF3108472B686
:1052F00013460A4601460348FCF780FE84F31088F3
:1053000010BD0000E800002013B50146012301AAEA
:105310000148FDF742F81CBDE800002010B5EFF38E
:10532000108472B613460A4601460348FDF735F865
:1053300084F3108810BD0000E800002070470000D2
:105340002DE9F04300228BB054A31146022001F056
:105350004BF90024022501260096CDE9015453A300
:1053600022462146284601F03FF90096CDE9015436
:10537000002257A31146022001F036F95D4B0022AE
:105380004FF47A715C48009401F0A2FA5A4801F097
:1053900041FB5B4859495F4D01605A4981605A4958
:1053A00041605A49C1605A49016129688847686962
:1053B0008047594F800DB860E968584888470022F7
:1053C00057A31146022001F00FF9002259A31146FC
:1053D000022001F009F97D20002200905AA3114615
:1053E000022001F001F94FF00A0800225BA31146E8
:1053F0000220CDF8008001F0F7F840F6B8300594AF
:105400000694CDE907404FF00809CDE90169CDF8D0
:105410000080CDE9034600231621D5F81CC01A46AA
:105420000120E047CDE90846CDE904460520069471
:105430000794CDE90204CDE9004901230A22AC69B1
:1054400000211846A047FF216A6D012090470120E6
:10545000FBF7BCF80220FBF7B9F80020FBF7B6F821
:1054600001210020FBF7ECF8FF214048FAF7F8FF94
:10547000B868012200903EA30021104601F0B4F864
:10548000B868696B00F6B83088470BB00021BDE8FA
:10549000F0433A4A012001F08DB900000A0D50494D
:1054A0004E4720504F4E470A0D0000004150504CCF
:1054B00049434154494F4E5F56455253494F4E3A26
:1054C000205625582E25582E25580D0A000000007C
:1054D0004D575F524144494F5F56455253494F4ED5
:1054E0003A202020205625582E25582E25580D0AC2
:1054F000000000000930000800040020A52F00086B
:10550000E4010020452E0008D52F0008712F000867
:10551000412F0008D470000818000020C0CA893646
:105520002D2D2D2D2D2D2D2D2D2D2D2D2D2D2D0ACE
:105530000D0000004C4F52415F4D4F44554C4154BB
:10554000494F4E0A0D0000004C4F52415F42573DFB
:105550002564206B487A0A0D000000004C4F524130
:105560005F53463D25640A0D00000000FF02002045
:1055700072616E643D25640A0D000000D1300008A0
:10558000704730B50024039D19442A4412B262F3D7
:105590000F04B2F57A7F04DBA2F57A7262F30F048E
:1055A000491CC0E9001430BD70B586B00446002027
:1055B0000D4D01900290296902A888470190E86882
:1055C000804760F30F0668688047014602980090A4
:1055D000324603A8019BFFF7D4FFDDE90301C4E9CC
:1055E000000106B070BD00001C6F000810B54FF040
:1055F000B040816821F40041816001F0E5F90B4978
:105600000120087001F04AF8094801F069F8022009
:1056100001F06CF801F08EF80121084601F092F8D3
:105620000121BDE81040084601F09EB800000020AE
:10563000C15A000810B59AB048216846FAF732FFFF
:10564000182112A8FAF72EFFFBF740FD4FF0B040EB
:1056500050F8901F21F0180101601648016821F4EC
:10566000C06141F4007101600068002400F4C06072
:10567000189024200090812003900120CDE9080497
:10568000B020CDE90A046846FBF7A4FF08B172B662
:10569000FEE74F20CDE912041494159416940221CC
:1056A00012A81794FBF70EFE002801D072B6FEE791
:1056B0001AB010BD00040058704700000148FCF704
:1056C00045BA0000B000002002210148FCF70ABAE8
:1056D000B000002000210148FCF704BAB00000200F
:1056E00001210148FCF7FEB9B0000020024602216A
:1056F0000148FCF7FDB90000B0000020024600217F
:105700000148FCF7F5B90000B00000200246012175
:105710000148FCF7EDB90000B00000204FF47A71A9
:10572000A0FB0110820542EA9120704710B5810D5F
:1057300080024FF47A720023FAF76CFD10BD70B549
:10574000FFF7F4FF0446FBF79FF8054600E000BFB3
:10575000FBF79AF8401BA042F9D370BD03207047B5
:1057600070B50446FBF790F80546FFF7ADFF002241
:10577000511950418B0A43EA8053C1F30900FFF7E6
:10578000CDFF2080184670BD01484068704700007A
:105790000400002010B5FBF777F802494968401A69
:1057A00010BD0000040000200349002009780029F2
:1057B00001D0FBF769B87047040000202DE9F041E3
:1057C0000E4D00272878B0B90D4E7C1E3463FDF7CE
:1057D000B1FA00F045F84FF480713046FCF714FA46
:1057E00030463463FCF78AF90020FFF77FFF00F0B2
:1057F00009F8012028703846BDE8F0810400002037
:10580000B000002010B5FBF73FF80149486010BD1B
:105810000400002030B58BB0044600252C216846DA
:10582000FAF740FE00F01CF80B4800210122406806
:1058300007912044C04301904FF00050CDE905107E
:1058400040150A9069460548FCF7AEFA08B1FBF727
:1058500018F80BB0284630BD04000020B00000202E
:1058600010B5064900240120086001020448FCF735
:10587000CBF90349601E0863204610BD5C28004038
:10588000B0000020F0B54FF0FF35EFF3108772B68F
:10589000134E4FF0000C4FF0010E738A328AC3F59D
:1058A000007493420BD3A4B2A0420AD3824208D917
:1058B00086F802E033801446A6F812C001E0D21A3E
:1058C00094B2844207D9728A0A80718A00250844FA
:1058D000C0F30800708287F310882846F0BD0000EE
:1058E000A4050020EFF3108072B6034AD18A491C48
:1058F000D18280F310887047A405002070B500267F
:10590000EFF3108472B61D4DE88A10B184F310884D
:105910002EE0FFF7E7FF288A698A88422AD0AA7812
:10592000012A01D072B115E02A88101A0004000C77
:10593000A8824FF00202AA704FF000022A8009D11B
:10594000AA702A82288A814201D9081A01E0C0F58A
:105950000070A8820949288A1831461884F31088F3
:1059600000F0BAFE0648A98AC2683046904706464B
:10597000304670BD00F050F8C8E70000A4050020D4
:10598000306F000870B5EFF3108172B6204C00251F
:10599000A078022814D0208AA28A1044C0F30800FC
:1059A0002082228A608A824202D0E38A012B0AD0B6
:1059B00081F3108800F08CFEBDE8704000F02CB838
:1059C000A5702582EDE7A378012B01D063B113E028
:1059D00023889A1A1204120CA2824FF00203A370B9
:1059E000258009D1A5702582228A904201D9801A8A
:1059F00001E0C2F50070A082054A208A18321044E6
:105A000081F31088034AA18AD268BDE8704010472C
:105A1000A4050020306F0008EFF3108072B6034A2F
:105A2000D18A491ED18280F310887047A4050020D6
:105A30000549096804E0814201D1012070474969A4
:105A40000029F8D10020704774000020044A116832
:105A500009B100230B724161106000F017B800001B
:105A600074000020084910B50A68516941B1036803
:105A70000C68A34201D90A46F7E75061416110BDA5
:105A800000215061FAE700007400002070B50B4D52
:105A90000446286A8047064601202072A86980478C
:105AA00021683044884201D8084603E0A86980474D
:105AB00030442060A968BDE870400847F06E0008D7
:105AC0003EB505460C4601A8FFF76EFDBDF908106E
:105AD000009105A210212846019B01F0E0F828461C
:105AE000FAF70FFC20803EBD256473253033643AFD
:105AF0000000000030B5416EB9B10268916892684B
:105B0000C1F342610B4C520FA35CDD0004F10803AA
:105B10009A5CB5FBF2F2A0F86A20625C595CD20094
:105B2000B2FBF1F1A0F8681030BD0121A0F86A10B5
:105B3000F8E70000746F000890F82810C90706D035
:105B400001684A68C36A22F400321A434A6090F836
:105B50002810890706D501684A68036B22F4803251
:105B60001A434A6090F82810490706D501684A6828
:105B7000436B22F480221A434A6090F828100907E8
:105B800006D501684A68836B22F400421A434A60D2
:105B900090F82810C90606D501688A68C36B22F4FC
:105BA00080521A438A6090F82810890606D5016849
:105BB0008A68036C22F400521A438A6090F8281015
:105BC000490611D501684A68436C22F480121A43D1
:105BD0004A60416CB1F5801F06D101684A68836C48
:105BE00022F4C0021A434A6090F82810090606D52C
:105BF00001684A68C06C22F4002202434A60704780
:105C0000F8B500250446C0F88C50FBF79DF907460F
:105C1000206800686FF07E46000708D53B460022EA
:105C20004FF400112046009600F076FC60B9206821
:105C3000006840070AD53B4600224FF48001204609
:105C4000009600F069FC08B10320F8BD2020C4F8DC
:105C50008400C4F8880044F86C5F00202575F8BD06
:105C600010B5806A0021A0F85E10A0F85610FCF76D
:105C7000A9FC10BD70B5846AD4F88400D4F88850AB
:105C8000216889684FF00006090606D5212804D14D
:105C9000A4F85660204600F065F820688068400649
:105CA00006D5222D04D1A4F85E60204600F030F81D
:105CB000D4F88C0040F01000C4F88C002046FCF7AB
:105CC00081FC70BD10B50146806A096809688906C3
:105CD00016D40021A0F856100168083151E8002FB1
:105CE00022F0800241E80023002BF5D1016851E841
:105CF000002F42F0400241E80023002BF6D110BDF6
:105D0000FCF71EFF10BD10B5806AFCF727FF10BD21
:105D100010B5016851E8002F22F4907241E8002389
:105D2000002BF6D10E4B0168083151E8002F1A40C4
:105D300041E80024002CF6D1C16E012908D1016888
:105D400051E8002F22F0100241E80023002BF6D189
:105D50002021C0F888100021C166016710BD000035
:105D6000FEFFFFEF016851E8002F22F0C00241E87A
:105D70000023002BF6D10168083151E8002F22F4EE
:105D8000000241E80023002BF5D12021C0F8841047
:105D9000704710B5B0F86020D0F888300168222B29
:105DA00004D0886940F00800886110BD496A836D9D
:105DB00011401980816D891C8165B0F85E10491E03
:105DC000A0F85E10B0F85E100029EED1016851E82D
:105DD000002F22F4907241E80023002BF6D10168D5
:105DE000083151E8002F22F0010241E80023002B86
:105DF000F5D12021C0F8881000210167C26E012A68
:105E000002D0FCF72FFE10BDC166016851E8002FDB
:105E100022F0100241E80023002BF6D10168CA6984
:105E2000D243D20601D410220A62B0F85C10FCF70B
:105E300034FB10BD2DE9F0470446B0F860900068CF
:105E4000C56907688668D4F88810222905D0816959
:105E500041F008018161BDE8F087B4F868804FF037
:105E6000000A61E02068406AA16D00EA090008802C
:105E7000A06D801CA065B4F85E00401EA4F85E0012
:105E80002068C56969072DD0E90709D0F90507D54C
:105E900001210162D4F88C0040F00100C4F88C00AC
:105EA000A8070AD5F00708D0216802200862D4F8B4
:105EB0008C0040F00400C4F88C0068070AD5F00795
:105EC00008D0216804200862D4F88C0040F0020059
:105ED000C4F88C00D4F88C0020B12046FCF772FB8B
:105EE000C4F88CA0B4F85E00F0B9206850E8001F38
:105EF00021F4807140E80012002AF6D1274A206878
:105F0000083050E8001F114040E80013002BF6D184
:105F10002020C4F88800C4F870A0E16E5046012922
:105F200025D02046FCF79EFDB8F1000F01D0A80651
:105F300098D4B4F85E0000288DD0B4F8681081427F
:105F400089D92068083050E8001F21F0805140E8CE
:105F50000012002AF5D112482067206850E8001F7F
:105F600041F0200140E80012002AF6D173E7E06614
:105F7000206850E8001F21F0100140E80012002ABC
:105F8000F6D12068C169C943C90601D41021016254
:105F9000B4F85C102046FCF780FAC5E7FEFFFFEF7F
:105FA000935D000810B5B0F86020D0F88830016823
:105FB000222B04D0886940F00800886110BD496A2E
:105FC0001140826D1170816D491C8165B0F85E10C1
:105FD000491EA0F85E10B0F85E100029EED10168ED
:105FE00051E8002F22F4907241E80023002BF6D1F3
:105FF0000168083151E8002F22F0010241E8002336
:10600000002BF5D12021C0F8881000210167C26E55
:10601000012A02D0FCF726FD10BDC166016851E8D7
:10602000002F22F0100241E80023002BF6D1016876
:10603000CA69D243D20601D410220A62B0F85C10B9
:10604000FCF72BFA10BD00002DE9F0470446B0F82C
:1060500060900068C56907688668D4F888102229AE
:1060600005D0816941F008018161BDE8F087B4F88D
:1060700068804FF0000A61E02068406AA16D00EA84
:1060800009000870A06D401CA065B4F85E00401EB9
:10609000A4F85E002068C56969072DD0E90709D01A
:1060A000F90507D501210162D4F88C0040F0010008
:1060B000C4F88C00A8070AD5F00708D02168022090
:1060C0000862D4F88C0040F00400C4F88C00680723
:1060D0000AD5F00708D0216804200862D4F88C00A3
:1060E00040F00200C4F88C00D4F88C0020B12046A7
:1060F000FCF768FAC4F88CA0B4F85E00F0B9206828
:1061000050E8001F21F4807140E80012002AF6D107
:10611000274A2068083050E8001F114040E800136B
:10612000002BF6D12020C4F88800C4F870A0E16EDE
:106130005046012925D02046FCF794FCB8F1000F09
:1061400001D0A80698D4B4F85E0000288DD0B4F829
:106150006810814289D92068083050E8001F21F07A
:10616000805140E80012002AF5D1124820672068CB
:1061700050E8001F41F0200140E80012002AF6D14B
:1061800073E7E066206850E8001F21F0100140E846
:106190000012002AF6D12068C169C943C90601D49A
:1061A00010210162B4F85C102046FCF776F9C5E7CF
:1061B000FEFFFFEFA55F00082DE9F04104460068EF
:1061C0002269A168E66911436269002532431143DF
:1061D000834B0268834E32400A4302602068416864
:1061E000E26821F44051114341602168A06999425D
:1061F00001D0226A10438A687B4E324002438A6093
:106200002068C16A626A21F00F011143C1627749B7
:1062100022684FF0B0408A4213D1D0F8880000F0D5
:10622000030040F44030B0F5403F08D06FF44031F7
:10623000401832D001282ED0022830D129E0012088
:106240002EE06B498A4213D1D0F8880000F00C0090
:1062500040F44020B0F5402F08D0001FB0F540209A
:106260001BD0042817D0082819D119E0002017E006
:106270009A4214D1D0F888004FF4406110F4406085
:106280000ED0B0F5806F08D0B0F5006F03D0884213
:1062900005D1082004E0022002E0042000E01020E4
:1062A0005449554E00274FF4004C9A4233D130B137
:1062B00002280DD0042805D008282BD107E0FBF7D1
:1062C000F7F801E0FBF714F9010001D17EE0614627
:1062D000606A36F810206668B1FBF2F006EB460300
:1062E00083426FD8B0EB063F6CD8002308461946AE
:1062F000F9F790FF090241EA1061020270081018D4
:10630000794132460023F9F785FF3C4AA0F54071F8
:10631000914259D956E0E2694FF6EF7862452DD1A6
:1063200009284FD2DFE800F00508114E0D4E4E4E01
:106330001000FBF7BDF801E0FBF7CAF8010004D13B
:1063400044E0FBF7D5F8F9E76146606A36F81000DB
:10635000B1FBF0F04100606801EB5001B1FBF0F0DF
:1063600080B2A0F1100141452CD84FF6F0710140E8
:10637000C0F3420001432068C16027E0092821D210
:10638000DFE800F0050811200D2020201000FBF7A9
:106390008FF801E0FBF79CF8010004D116E0FBF751
:1063A000A7F8F9E76146606A36F81000B1FBF0F132
:1063B000606801EB5001B1FBF0F080B2A0F1100178
:1063C000414501D9012501E02168C8600120A4F8F8
:1063D0006A0024F8680F2846A760E760BDE8F081EE
:1063E00000800040F369FFCFFFF4FF110038014047
:1063F000004400400024F4005C6F0008FFFC0F0024
:1064000070B58165A0F85C20A0F85E2000240467C8
:1064100081684FF48055FF23A94204D10169F9B97D
:1064200040F2FF1122E07F26C1B1B1F1805F1AD0A6
:10643000A0F86040C0F88C402221C0F888100168A4
:10644000083151E8003F43F0010341E80036002ED7
:10645000F5D1416EB1F1005F0ED032E0016941B972
:10646000A0F86030E6E7016919B13F21A0F860109B
:10647000E0E7A0F86060DDE7B0F86810914220D84E
:106480008168A94201D10169C9B11F49016780F83A
:106490008040016941B1016851E8002F42F48072E7
:1064A00041E80023002BF6D10168083151E8002FA4
:1064B00042F0805241E80023002BF5D121E013493E
:1064C000E4E78168A94201D1016979B11049016706
:1064D00080F88040016959B1016851E8002F42F409
:1064E000907241E80023002BF6D10AE00949EEE75B
:1064F000016851E8002F42F0200241E80023002B00
:10650000F6D1002070BD000049600008355E00082B
:10651000A55F0008935D00082DE9F0471F469046EF
:106520000E4604464FF0000A4FF02009089D49E04E
:10653000681C47D0FAF708FDC01BA8422AD84DB303
:106540002068016849073DD5C069C043000539D4BA
:1065500021684FF400600862206850E8001F21F4B1
:10656000D07140E80012002AF6D12068083050E8C7
:10657000001F21F0010140E80012002AF5D144F883
:10658000849FC4F80490C4F8089004F804AC032075
:10659000BDE8F087206850E8001F21F4D07140E882
:1065A0000012002AF6D12068083050E8001F21F0C0
:1065B000010140E80012002AF5D144F8849FC4F894
:1065C0000490E2E72068C06936EA000004D00020A9
:1065D0004045ADD00020DBE70120F9E70148FBF79B
:1065E000F3BF0000F40000200FB4002370B586B0A4
:1065F000ADF81030274B1C7A844205D26FF00400AE
:1066000006B070BC5DF814FBD868814302D06FF00F
:106610000500F5E75B681BB112B104A9684698470D
:106620000EAB4FF480751C4629461B480D9A00F0AE
:106630003FFB0646FFF756F9BDF8100005A93044A8
:1066400080B2FFF71FF9401C1ED0124900201831FC
:106650006B4608E0BDF814201E5C8E54521C401C92
:10666000ADF8142080B2BDF810209042F2D3BDF8EE
:1066700014002346084429460D9A00F019FBFFF741
:10668000CBF9FFF73BF9BBE7FFF7C6F96FF0020064
:10669000B6E70000A4050020BC07002010B51822B2
:1066A0000021084800F07BF806484FF400720021F2
:1066B000183000F074F804480168BDE81040034841
:1066C00008470000A4050020306F00088559000825
:1066D0000021022000F048B80121022000F044B857
:1066E0000149486070470000A40500200149087274
:1066F00070470000A405002070B5EFF3108572B656
:106700000A480B4C016819B120688047606808E0AE
:10671000406818B1A0688047E06802E020698047BF
:106720006069804785F3108870BD00007800002004
:10673000D86E0008024800210160416070470000E7
:1067400078000020EFF3108272B6064B21B10129C8
:1067500005D15968014301E059688143596082F3CA
:10676000108870477800002010B5EFF3108472B6DF
:10677000054B1A6819B1012903D1024300E0824395
:106780001A6084F3108810BD7800002003E011F82F
:10679000013B00F8013B521E92B2F8D2704701E073
:1067A00000F8011B521E92B2FAD27047FFF7A4BF45
:1067B0007047704710B51446EFF3108372B6FDF7BB
:1067C000A9FF034941F8204083F3108810BD000061
:1067D000680000202DE9F047324D69688846014085
:1067E00069606869AB682968EF684FF0FF3605F1AA
:1067F0001C044FF0010934E00020114000E0401C6F
:1068000054F830200A42FAD054F8302004EBC00388
:106810000A405868104200D15E6058681040FDF789
:1068200079FF2861596809FA00F7B9435960EFF315
:10683000108C72B66969B9436961012104EBC10228
:1068400052F8083DBB431360491EF7D18CF3108802
:106850001449183151F8200080476869AB682968ED
:10686000EF686A680840104201D03B42C4D02E61F4
:10687000FFF79FFFEFF3108472B66A69A868296872
:106880000A4069680A4204D1E968084201D1FFF769
:106890008DFF84F31088FFF78BFFC5F80480BDE8F7
:1068A000F08700005000002010B5EFF3108272B6A0
:1068B000064B5C6904435C611C3353F8314004436C
:1068C00043F8314082F3108810BD000050000020D2
:1068D0002DE9F0411E46DDF818801746040011D05E
:1068E00086B1094800252560426A084690476060E5
:1068F00025726572A572C4E90368E77200206561BC
:10690000BDE8F0810120FBE7F06E000810B5034CF4
:10691000E0698047A16ABDE810400847F06E0008B2
:1069200070B5064C0646E06980470546616A304608
:106930008847281AA16ABDE870400847F06E000831
:106940002DE9F041EFF3108872B61D4F786980474A
:106950000446386980471B4E021B306860B300252F
:106960000168914202D9891A016000E0056040691E
:106970000028F5D10FE034686069306025726572D7
:10698000D4E903108847E07A012804D1A07A10B92D
:10699000204600F03FF8306870B100680028EAD067
:1069A000B8698047316809688842E4D8306818B10E
:1069B000017A09B9FFF76AF888F31088BDE8F08119
:1069C000F06E0008740000200249002008600248B0
:1069D0000068004774000020F06E000870B50500E4
:1069E0004FF0000411D00A48426A08469047686098
:1069F0002846FFF71DF830B1284600F049F8284630
:106A000000F008F80446204670BD0124FBE70000B2
:106A1000F06E00082DE9F04104004FF0000805D0A9
:106A20002046FFF705F808B9607A20B14FF0010859
:106A30004046BDE8F081EFF3108772B6124E6568EC
:106A4000306A8047854200D20546002025602072CA
:106A500001210E4D6172A072286860B1B069804753
:106A600021680844206029680968884206D22046C7
:106A7000FEF7ECFF05E030698047F8E72046FEF7B7
:106A8000F1FF87F31088D3E7F06E00087400002050
:106A900070B5002340B3EFF3108472B6144D4FF07D
:106AA0000106296886720A001BD0002646720B4632
:106AB000814213D10E72586918B12860FEF7E6FFC3
:106AC0000EE00C48C06880472E6009E0814203D187
:106AD00048695061002803E00A4649690029F5D158
:106AE000002384F3108800E00123184670BD0000E5
:106AF00074000020F06E0008FEE70907090E002868
:106B000004DB00F1E02080F80014704700F00F0073
:106B100000F1E02080F8141D704700002DE9F04FCF
:106B200091B0394CDDE91B57DDF868A0D4F800902E
:106B30007E0601D5D4F804909C1E232C03D300209C
:106B400011B0BDE8F08FFC0701D0302400E0202414
:106B5000A3460026BC0705D5002A03DA2D2652429B
:106B6000AAF1010A0024EE46B2B1B2FBF3FC03FB2A
:106B70001C28B2FBF3F219F808800EF80480641C9C
:106B8000002AF2D1AC4200DD2546AAEB0502FF0740
:106B90004FF0200309D00CE030228DF800200124B2
:106BA000F0E700F8013B491ECAD0171EA2F101020E
:106BB000F7DC36B100F8016B01E000F801BB491EBB
:106BC000BED0161EA2F10102F7DC30262F466D1E44
:106BD000A7420ADD00F8016B491EF7D1B0E72E5D30
:106BE00000F8016B491E01D1AAE77546261EA4F1E3
:106BF0000104F4DC03E000F8013B491EA0D0141EA0
:106C0000A2F10102F7DC9BE748000020FAF7A6F9A1
:106C1000FEF710FDFCF758F8FCF7D2F8FCF7D7F8B0
:106C2000FCE7F0B500242346264604E0CD5CED43A6
:106C3000CD54C6545B1C9342F8DB002321E0DD17E2
:106C400003EB557525F007069E1BC5F3C70CC6F16F
:106C500007075D1CEE1705EB567626F0070EA5EB31
:106C60000E05C5F1070EC6F3C70511F80C60FE400E
:106C700006F001067440465D04FA0EF73E434655A1
:106C80005B1CB3EBC20FDADBE10141EA841324B1F0
:106C9000002143EA41118154F0BD0121F9E70FB40D
:106CA00010B505AB049A00F003F810BC5DF814FBB6
:106CB0002DE9FE4F1F461546B1F1000B814602DC5F
:106CC0000020BDE8FE8F4C46ABF1010A86E0A4EB44
:106CD000090252456DDA252802D004F8010B7CE048
:106CE00015F8010F0021302800D101214FF0FF32AB
:106CF0003038164609280ED800266FF02F002B4694
:106D000006EB86061B7800EB46061E4415F8013F8D
:106D1000303B092BF3D928780A23692845D006DCB3
:106D200058283ED0632819D0642806D13DE0732846
:106D30001BD0752843D0782835D0252802D02520AF
:106D400004F8010BA4EB090CD44538DA287878B3A1
:106D500004F8010B2FE004F8010B00E02020761E60
:106D6000002EF8DC17F8040BB7E701CF5FEA000844
:106D7000404601D120A08046F9F7C3FA0146202001
:106D800001E004F8010B3246761E8A42F9DC00204D
:106D900004E018F8012B04F8012B401C8842F8DBB2
:106DA0001BE041F04001102309E041F0020106E040
:106DB00000E01CE06D1EA4EB090CD4450DDB01CFF7
:106DC0000096CDE90121A4EB0902ABEB02010246DA
:106DD0002046491EFFF7A2FE04466D1C28780028B5
:106DE0007FF475AFA4EB09025245BFF670AF0020E7
:106DF0002070A4EB090064E73C4E554C4C3E00006B
:106E000010B54FF0B040816B41F400318163816B6C
:106E100021F4003181630448FBF77CFD0F20FAF771
:106E2000B6F8002010BD0000F4000020064910B59F
:106E30004860FBF738FFFBF7CFFF0448016841F0DB
:106E400000610160002010BD0C0000208008005887
:106E50000F4910B588604FF400110E48FBF76BFB2B
:106E60000C480068C169C943C903FBD5C169C9435E
:106E70004902FBD4816841F4800181600548FBF739
:106E8000F5FA012202490348FBF7C2FD002010BDBC
:106E90000C000020F400002010B50848FBF704FDAA
:106EA00008B1F9F7EEFC0648F9F728FE002803D0F0
:106EB000BDE81040F9F7E5BC10BD0000F40000206B
:106EC000840100200A4610B501460248FBF7E6FDA2
:106ED000002010BDF40000208F300008BB300008F7
:106EE000A1300008BF3000088D300008B93000081C
:106EF000BD57000800000000155800086158000840
:106F0000055800088957000895570008A957000838
:106F10005D5700082D5700081D570008FD56000852
:106F2000D55600080D570008E156000861570008C3
:106F30002D6E0008016E0008516E0008C56E000835
:106F4000120024003000000006000C0010000000B9
:106F5000000000000100000002000000010002002B
:106F60000400060008000A000C0010002000400089
:106F70008000000101010103070100000804020470
:106F800008010101010000000300000005000000ED
:106F90000100000001000000060000000A000000DF
:106FA00020000000020000000400000008000000B3
:106FB0001000000040000000800000000001000000
:106FC00000020000A0860100400D0300801A0600A8
:106FD00000350C0040420F0080841E0000093D0077
:106FE00000127A000024F40000366E010048E80127
:106FF000006CDC0200000000000000000000000047
:107000000000000000000000000000000000000080
:10701000000000000100000002000000030000006A
:1070200004000000C01200001F000000A8160000AD
:1070300017000000841C00000F000000E425000081
:107040001E000000B42D00001600000008390000EA
:107050000E0000002C4C00001D000000685B0000CA
:1070600015000000747200000D0000005898000028
:107070001C00000034B7000014000000E8E4000029
:107080000C000000783101001B000000686E010058
:107090001300000034CA01000B0000002862020047
:1070A0001A00000040DB0200120000003C930300C5
:1070B0000A000000C0C204001900000060B305000F
:1070C00011000000382007000900000020A107007F
:1070D000000000002D350008FF340008B53B000813
:1070E0007D3B00087938000841390008393C000828
:1070F0004941000881340008D1450008253A0008BC
:1071000091450008A345000865390008A945000815
:10711000C94200085F390008E546000857390008F1
:10712000E94600085B390008813B0008013C000883
:1071300021350008BD350008C5390008E93E0008C2
:10714000B5460008A1460008213F00080543000895
:10715000B3330008A133000804050604030202014A
:1071600001010100000000000000000006070A0005
:1071700020001000080001000200100000000016AE
:107180000100001604000016303132333435363732
:1071900038394142434445464748494A4B4C4D4E95
:1071A0004F505152535455565758595A00000000E9
:1071B000303132333435363738396162636465666D
:1071C0006768696A6B6C6D6E6F70717273747576D7
:1071D0007778797A00000000F8710008000000203C
:1071E000B000000074010008A8720008B000002080
:1071F000881200009001000800000000000000005C
:10720000000000000000000000000000000000007E
:10721000000000010000000000000000010000006C
:10722000100000000000000000093D000000000008
:107230000000000000000000FF000000000000004F
:10724000B071000888710008FFFFFFFFFFFFFFFF1C
:10725000000000000000000000000000000000002E
:10726000000000000000000000000000000000001E
:107270000000000000000000000400480004004876
:1072800000040048000000480000004800000048DA
:107290009B070008A5070008AF0700080E000000C4
:0872A0000E0000000E000000CA
:0400000508000139B5
:00000001FF
